:1050000002FE2002FE6402F9A302FE2602FE6802EE
:10501000FE3D02FE6C02FE2302FE7002FE7402FEE2
:0D5020007802FE7C025100024500020000F3
:10502D00CD30E11520E00FC083C08288828C83CD06
:0C503D00F0D082D08322CDF222CDF622EA
:10504900CB30E11520E00FC083C08289828A83CBEF
:0C505900F0D082D08322CBF322CBF722D0
:10506500ED30E11320E00EC083C08288828C83E09E
:10507500D082D08322E2226405700EC083C082886C
:0B508500828C8393D082D08322E6222D
:10509000EB30E11320E00EC083C08289828A83E076
:1050A000D082D08322E3226405700EC083C082893F
:0B50B000828A8393D082D08322E72203
:0450BB00114901BFD7
:0650BF0009B900010A22FC
:0650C50029F9E43AFA2289
:0950CB00E0A3FBE0A3FAE0F922E6
:0950D4007401F5F0E025F0F02272
:0950DD00E0FBA3E0FAA3E0F922D4
:0950E600E0FDA3E0FCA3E0F822C8
:0150EF00229E
:1050F000EF64204E7005E4FE7F0122E4FE7F012272
:10510000D24112616C1200937B057A5D7954125979
:0C51100000E49043BEF02037030251A3DE
:10511C001200937B057A5D796A125900D218128BB2
:10512C00727F02128D14E49043BDF0128266EF6020
:01513C001260
:10513D009043BDE004F07B057A5D7984125900122D
:08514D000093128292EF601240
:105155009043BDE004F07B057A5D79991259001200
:0851650000939043BDE0701CB3
:10516D00D219128BBFD231D21A7F22128CEC1200BF
:0C517D00937B057A5D79AE125900801A10
:10518900C219128BBFC231C21A7F22128CEC1200D3
:10519900937B057A5D79C01259001282BABF00016A
:0351A900D34013DD
:1051AC001200937B057A5D79D3125900120093C2D9
:0351BC0008801E4A
:1051BF00120093904387E0FBE4C0E0EBC0E07B0577
:1051CF007A5D79EF12590015811581120093D2C5BE
:0551DF00E49043BDF067
:1051E400D2C5C2C59043BDE004F0B414F3120093D9
:1051F4007B057A5E7902125900120093D2AA12003A
:10520400937B057A5E7911125900E49043BDF0F561
:0952140048C24130070302548333
:06521D0012009620400C77
:0352230020FF0960
:0C5226007F11E4FD128FF4D24030400CE8
:0352320030FF0941
:0C5235007F12E4FD128FF4C240303735C8
:0952410030FD06302F032031116D
:03524A00303029D8
:0E524D00C219128BBF7F13E4FD128FF4801B79
:0C525B0030FD18302F1520301230310FBC
:0352670020300CE8
:0F526A00D219128BBF7F14E4FD128FF4302D0B7D
:05527900C22D303606D5
:0F527E00127D2C127AE91200962000030253D7FA
:10528D00C200127AB375F00A904294E084E5F0649E
:10529D00057002D22E75F005904294E084E5F0641D
:0352AD0002706F1D
:1052B000904D39E030E20312849E303E62904D39C9
:0552C000E05420605ADB
:0352C50030371A65
:1052C800128266EF60077F10E4FD128FF41282925B
:0D52D800EF60077F0FE4FD128FF430381AED
:1052E5001281F0EF60077F0DE4FD128FF4128179D2
:1052F500EF60077F0EE4FD128FF430360D128055F6
:10530500EF60077F0CE4FD128FF4303B0D128081B6
:10531500EF60077F0BE4FD128FF49043BEE0B40A03
:105325000050069043BEE004F09043BEE0B4032075
:10533500AD497C007E01E4FF1254A88E4A8F4BAD27
:105345004C7C007E01E4FF1254A88E4D8F4E8016D2
:10535500794AE4FA7B01AD4912FE80794DE4FA7B86
:1053650001AD4C12FE80E549B428004017E549B46B
:10537500B901D3500FE54CB40D004008E54CB450CD
:1053850001D34009C21A7F11128CEC8007D21A7F13
:0C53950011128CECE4F549F54C30253683
:1053A100120093904294E0FBE4C0E0EBC0E0904235
:1053B10095E0FBE4C0E0EBC0E0904296E0FBE4C086
:1053C100E0EBC0E07B057A5E791412590074FA258E
:1053D10081F581120093120096128F4990417EE06F
:1053E100FF1200A8EF9043BDF064486004E0B4569A
:0153F10018A3
:1053F20090417FE0FF1200A8EF9043BDF06453603C
:0554020004E0B44303C7
:105407001294809043BDE0645A6004E0B43F0312F5
:055417009480304244C6
:07541C0090417EE0B41B3D4E
:1054230090417FE09043BDF0B44100400F9043BDF5
:10543300E0B44401D3500512948080219043BDE031
:03544300B45B1A3D
:10544600904180E09043BDF0B44100400D9043BDD3
:10545600E0B44401D350031294802004030252178F
:10546600E5309043B5F0E5319043B6F0E532904330
:10547600B7F012008D12EB5CC20402521775D7000A
:1054860075A89075A70075D80075E8007597007522
:03549600C8002229
:0A549900E0C0E0A3E0F582D083221A
:1054A300E0A3FEE0FFEF8DF0A4CFC5F0CCA42CFC6D
:0954B300EE60038DF0A42CFE2232
:1054BC00C2D1C2D5EE30E707D2D1D2D5125569ECA4
:1054CC0030E705B2D11255711254E430D1031255A4
:1054DC006930D50312557122BC000EBE0032EF8D1F
:1054EC00F08420D226FFADF0227B0075F008EF2F60
:1054FC00FFEE33FEEB33FBEE9DEB9C4005FBEE9D8C
:10550C00FE0FD5F0E9E4CECDCBCC227EFF7FFF227F
:10551C00EDB410005022EE8DF084FEEF54F045F007
:10552C00C48DF084C4FCEF540FC445F0C48DF084DA
:10553C00FFADF0E4CC4FFF22EE8DF08420D2CC7E78
:10554C0008CEC5F0CDCBEF2FFFED33FD10D7079B69
:10555C005005D5F0F1229BFD0FD5F0EA22C3E49F54
:0D556C00FFE49EFE22C3E49DFDE49CFC22B2
:10557900EB700122E8FEE58124FDF8E6C0E008E6CB
:10558900C0E0EEF8125721D0E0158129F8E43AFC81
:10559900EB54072390559F7380068007800C800089
:0D55A900E4F6228C838882E4F022E4F222F2
:1055B600D2D57F018002C2D5ED700302571C540775
:1055C6002323F58289F0EAFDEB700122540345821C
:1055D6002390562073E608F70920D50470F7803F1C
:1055E600DEF3DFF1803989828D83E608F0A320D5CA
:1055F6000470F7802ADEF3DFF18024E608F3092041
:10560600D50470F78019DEF3DFF1801388828C836E
:10561600E0A3F70920D50470F78004DEF3DFF1027A
:10562600571980B180AF80BE80D180E080DE805186
:10563600806B80168014803480218099809780A6A4
:1056460080B980438041803C8068E208F70920D514
:105656000470F780CADEF3DFF180C4E208F30920A4
:10566600D50470F780B9DEF3DFF180B389828D83CC
:10567600E208F0A320D50470F780A4DEF3DFF18002
:105686009E0256F40256CE88828C83E493A3F709D1
:1056960020D50470F68088DEF2DFF080F888828CF0
:1056A60083E0A3F30920D50470F780E9DEF3DFF188
:1056B60080E388828C83E493A3F30920D50470F6F3
:1056C60080D3DEF2DFF080CD88828C83E493A3C999
:1056D600C582C9CDC583CDF0A3C9C582C9CDC58351
:1056E600CD20D50470E680ADDEE2DFE080A78882BB
:1056F6008C83E0A3C9C582C9CDC583CDF0A3C9C536
:1057060082C9CDC583CD20D50470E780DFDEE3DF17
:03571600E180D956
:08571900A9F022E4FBFAF922D9
:10572100D2D5E8C0E0E58124FCF8E6FF08E6FE4FAB
:105731007005D0E00257190FBE00011FD0E0F8023A
:0257410055BE53
:10574300EBFDEAFCE9F8125090B42005E4FE7F017A
:0657530022E4FE7F0122AA
:10575900EBFDEAFCE9F8125090B42005E4FE7F0164
:0657690022E4FE7F012294
:10576F00EBFDEAFCE9F8125090B42005E4FE7F014E
:06577F0022E4FE7F01227E
:10578500EBFDEAFCE9F8125090B42005E4FE7F0138
:0657950022E4FE7F012268
:10579B00EBFDEAFCE9F8125090B42005E4FE7F0122
:0657AB0022E4FE7F012252
:1057B100EBFDEAFCE9F8125090B42005E4FE7F010C
:0657C10022E4FE7F01223C
:1057C700EBFDEAFCE9F8125090B42005E4FE7F01F6
:0657D70022E4FE7F012226
:1057DD00EBFDEAFCE9F8125090B42005E4FE7F01E0
:0657ED0022E4FE7F012210
:1057F300EBFDEAFCE9F8125090B42005E4FE7F01CA
:0658030022E4FE7F0122F9
:10580900EBFDEAFCE9F8125090B42005E4FE7F01B3
:0658190022E4FE7F0122E3
:10581F00904453EBF0A3EAF0A3E9F0904456EDF077
:10582F00A3ECF0A3E8F0125065F5F0125090B5F02C
:0B583F0005E4FE7F0122E4FE7F012251
:10584A00EBFDEAFCE9F8125090B42005E4F9FBFA02
:06585A0022E4FBFAF92232
:10586000EBFDEAFCE9F8125090B42005E4FE7F015C
:0658700022E4FE7F01228C
:09587600BF2003E4FF22E4FF223D
:10587F00EF64204E7005E4FE7F0122E4FE7F0122DB
:10588F00904459ECF0A3EDF0ECFAEDF9125090FDC5
:10589F003395E0F5F0E4B5F00B8DF0EFB5F005E4DE
:0958AF00FE7F0122E4FE7F0122CC
:1058B80090445BECF0A3EDF0ECFAEDF9125090FD9A
:1058C8003395E0F5F0E4B5F00B8DF0EFB5F005E4B5
:0958D800FE7F0122E4FE7F0122A3
:0158E10022A4
:0158E20022A3
:0158E30022A2
:0758E400BF2002D322D322F2
:0758EB00BF2002D322D322EB
:0758F200BF2002D322D322E4
:0758F900BF2002D322D322DD
:10590000A881058118EBC6C908CAC6CA08F67BFF7C
:10591000312ED0E0D0E0D0E0C082C08322D083D04E
:1059200082EDC0E0ECC0E0E8C0E0C082C083E58169
:10593000F8241EF58108E8C9CBF709EAF709EBF767
:1059400009770009E924F6FA75F000C2D5E924FCCC
:10595000F8E924F9F9ECC0E0E8C0E091971250654D
:10596000FFE92409F9D0E0F8D0E0FCEF605020D541
:1059700074B4250AE4FB74FFFCF7D2D580D391B050
:1059800080CFFF20F71CBCFF067014D2F380C2EC5E
:10599000C0F075F00AA42FD0F030F703F78001FCB7
:1059A00080AFB7FF03EF80F4E780E57F0091B01987
:1059B0001709800DEF24D0B40A0040C68093B6FFCB
:1059C000EAE581C3941AF581E4FED0E0FFD082D0ED
:1059D00083D0E004600ED083D082158115811581BB
:1059E000C082C08322905CEBE49360256FA36006C5
:1059F000A350F5A380F293FF400442F080BEE4A3DD
:105A0000938F83F582E4C2D130F705B7FF027700A8
:105A10007340A1D3A380D1EAC8FDE620F703FC8040
:105A200001F71A1AEDF88094D2D17F7880027F585E
:105A3000912B90100441C3BCFF028054C0F08AF047
:105A4000EAC92419F583E8FEECC0E091971250658D
:105A5000FF601AC583C9C583F70B19E9C583F90827
:105A6000B800010CEE2404F9E7C39B70E0D0E0FC21
:105A7000E5F024FDFAD0F08B82A98309EEC394FBF4
:105A8000F583F8E7F60809D582F9A9831819614D5D
:105A90008AF0EAC9F583E8FE9197125065FF60131A
:105AA000EEC8CE8D8291B0AD82EEC8CE08B800EAC5
:105AB0000C80E7A983E5F024FDFA21487F30912B83
:105AC000900806C2F7913BE8CAC9C88055D2F7EAE8
:105AD000147D0230F4047D0424FEF8E68A83A88352
:105AE00030E70DD2D1C3E496F618DDFAA883800022
:105AF000C2F7912B900A05913BC9C8CAC9C2F07F71
:105B00002D20D10530F5047F2BD2F08015912BE6A6
:105B100018188004912B7425C2F7F70BCAC9C8CA9C
:105B2000C2F0E7FDE924002BF8B6300318DBFABB1E
:105B300000080B08BD00031B8013BDFF02800EEDA3
:105B4000C39BFE4008600674307195EDFBEB70025C
:105B50002148EC046023D39B401F601DFE7D202064
:105B6000F13830F3027D3030F023BD3018719118D8
:105B7000EF30E60118910F804030F03F910F0B306D
:105B8000F6390B8036EF910F1E30F6011E719180B1
:105B900028EE6005ED08F6DEFC2230F007910F0BD1
:105BA00030F6010BE9FF2419F9E6F71918DBFAEDD5
:105BB000F719DEFCEFF92419F8CCCB1919E8C0E08D
:105BC000E6FF91970909EF911CD0E0F818DBEE0988
:105BD0000921481A1A9133905CDFE6086002240616
:105BE000936023F7190B30E504E4A380F3EBC0E0E6
:105BF000743AF7E924FCF908901004913B18D0E0BE
:105C00002405FBE92404C8CAC9E92419F880AC08B2
:105C1000EFF68FF030F604743008F622BDFF05125F
:105C2000006C800312502D09071922E9CAC8E92423
:105C300001F922E9CAC8E92419F922A2F492D5C0CF
:105C4000F0E582FD30D50623F582FD181818E685AB
:105C500083F084F620D5047B0180027B0308E5F005
:105C6000D6C6C48583F084C4C6C445F0C48583F019
:105C700084D6DBE9E5F024F6500730D10224202455
:105C800007243AF70920D509DDC3D0F01818AB82F4
:105C900022DDB8181880F3E7F819E7FC19E7FDBD15
:105CA000FF0122090907B70004190719221919224F
:105CB000CACDE8C0E0E9C0E0E6FB08E6FA08E6F98C
:105CC000EFBBFF0512006C800A06B6000318060839
:105CD000125049080618D0E0F9D0E0F8CDCA2228C1
:105CE0006E756C6C290049584450434C046C10622A
:105CF00000680023012D022B2020402E80002A5A0C
:015D0000178B
:105D01006F5ABC785A28585A2E735A37755AF0640C
:0F5D11005ACD695ACD635B0D255B14705BD300CF
:105D200090445DECF0A3EDF0ECFAEDF9125090FD2B
:105D30003395E0F5F0E4B5F00B8DF0EFB5F005E448
:095D4000FE7F0122E4FE7F012236
:095D4900BF2003E4FF22E4FF2265
:025D520000DD72
:105D540046696E6973686564204D61696E20496E99
:105D6400697420210A0020202020204465666C6587
:105D74006374696F6E20456E61626C6520210A0050
:105D84002020202020202048204465666C204F6677
:105D94006620210A0020202020202020562044654F
:105DA400666C204F666620210A00202020202048AF
:105DB4005620456E61626C6520210A002020202057
:105DC4002048562044697361626C6520210A00559D
:105DD40073696E6720436F6E6669672030202844BC
:105DE400656661756C742920210A005573696E67B4
:105DF40020436F6E66696720256420210A0050469F
:105E04005720456E61626C656420210A00230A00F4
:105E1400253032643A253032643A25303264202108
:025E24000A0072
:105E26005374617274696E67204D61696E204669AC
:105E3600726D7761726520210A0053746172746510
:105E46006420543220210A00496E697469616C69C4
:105E56007A696E672049324320636F6E74726F6C85
:105E66006C657220210A0020202020202B435055EB
:105E7600204C6564202D2061646472203438202112
:105E86000A00693263207772697465206661696CFD
:105E9600210A0020202020202D435055204C6564E7
:105EA600202D206164647220343820210A002020CD
:105EB6002020202B566964656F20505741202D20E5
:105EC6006164647220393420210A002020202020B9
:105ED6002D566964656F20505741202D20616464FA
:105EE6007220393420210A0020202020202B4465EE
:105EF600666C656374696F6E20505741202D206172
:105F060064647220394320210A00202020202020AA
:105F160020202B204E2D5320436F727265637469C7
:105F26006F6E202D206164647220353420210A00B2
:105F360020202020202020202D204E2D5320436F6E
:105F46007272656374696F6E202D206164647220BD
:105F5600353420210A0020202020202D4465666C3F
:105F6600656374696F6E20505741202D206164640B
:105F76007220394320210A0020202020202B436F45
:105F86006E76657267656E636520505741202D20D9
:105F96006164647220344620210A002020202020DB
:105FA6002D436F6E76657267656E63652050574147
:105FB600202D206164647220344620210A002020AE
:105FC6002020202B4C56505320505741202D206125
:105FD60064647220393620210A0020202020202DDA
:105FE6004C56505320505741202D20616464722036
:105FF600393620210A0020202020202B473220502D
:106006005741202D206164647220413520210A0009
:1060160020202020202D473220505741202D20615E
:1060260064647220413520210A0020202020202B84
:106036004856204D6F6E202D2061646472203932DF
:1060460020210A0020202020202D4856204D6F6E4A
:10605600202D206164647220393220210A0020201C
:106066002020202B566964656F204D697865722063
:10607600505741202D206164647220343620210A55
:106086000020202020202D566964656F204D6978F8
:10609600657220505741202D206164647220343689
:1060A60020210A006661696C656420746F2074752E
:1060B600726E206F6E20636F6E76657267656E63B3
:1060C6006520210A0077617374655F696478203DF5
:1060D60020253032582C2073657474696E672074DD
:1060E6006F20300A00777269746520656570726F7B
:1060F6006D206661696C6564207570646174696E93
:10610600672077617374655F69647821200A007778
:106116007269746520656570726F6D206661696C61
:106126006564207570646174696E67206F7065724E
:106136006174696E672074696D65210A00777269FA
:10614600746520656570726F6D206661696C656443
:10615600207570646174696E672077617374655F1A
:06616600696478210A00C3
:10616C0075A61E75A6E11200937B057A5E79261240
:10617C005900120093120093C20075516475C90046
:10618C0075C80475CD0075CC00D2BDD2AD75CBDC15
:10619C0075CA00E4904294F0904295F0904296F0CB
:1061AC00904297F0A3F01200937B057A5E7940122F
:1061BC005900C234E4F548C23FC240904276F0C266
:1061CC0042904277F075B0FF75F8FFD288D28AD230
:1061DC00A8F5C675A704120096E4904387F0C23365
:1061EC00D23E759710E5A74480F5A7120096E4906F
:0361FC0043C2F0AB
:1061FF00E49043C0F0E49043C1F09043C1E0B40891
:07620F0001D340030262A667
:106216001200969043C1E0FBE4C0E0EBC0E090437F
:10622600C0E075F009A4FD9043C2E075F077A424A0
:1062360057F582E4344CF583ED2582F582E4358307
:10624600F583D0E02582F582D0E03583F583E0C082
:10625600E09043C1E0FDE4C0E0EDC0E09043C0E063
:1062660075F009A4FFE4C0E0EFC0E09043C2E0751A
:10627600F077A424C5F582E43442F583D0E0258284
:10628600F582D0E03583F583D0E02582F582D0E033
:106296003583F583D0E0F09043C1E004F002620953
:1062A6009043C0E004F0B405028003026204E4F007
:0562B600E49043C1F07B
:1062BB001200969043C1E0FBE4C0E0EBC0E09043DA
:1062CB00C0E02323FD9043C2E075F077A42484F54E
:1062DB0082E4344CF583ED2582F582E43583F58336
:1062EB00D0E02582F582D0E03583F583E0C0E090E5
:1062FB0043C1E0FDE4C0E0EDC0E09043C0E02323E8
:10630B00FFE4C0E0EFC0E09043C2E075F077A42457
:10631B00F2F582E43442F583D0E02582F582D0E0B9
:10632B003583F583D0E02582F582D0E03583F58384
:10633B00D0E0F09043C1E004F0B4040280030262A9
:10634B00BB9043C0E004F0B4060280030262B69037
:10635B0043C2E075F077A4242BF582E4344CF5832B
:10636B00E0FC9043C2E075F077A4FB2499F582E43E
:10637B003442F583ECF0EB242CF582E4344CF583BA
:10638B00E0FD9043C2E075F077A4FB249AF582E41C
:10639B003442F583EDF0EB242DF582E4344CF58398
:1063AB00E0FCA3E0FD9043C2E075F077A4FB249BD7
:1063BB00F582E43442F583ECF0A3EDF0EB242FF5FA
:1063CB0082E4344CF583E0FCA3E0FD9043C2E0751E
:1063DB00F077A4FB249DF582E43442F583ECF0A323
:1063EB00EDF0EB2431F582E4344CF583E0FC904383
:1063FB00C2E075F077A4249FF582E43442F583EC78
:10640B00F0120096E49043C0F09043C0E0FF90433D
:10641B00C2E075F077A42437F582E4344CF583EFB2
:10642B002582F582E43583F583E0C0E09043C0E03C
:10643B00FDE4C0E0EDC0E09043C2E075F077A4242A
:10644B00A5F582E43442F583D0E02582F582D0E0D5
:10645B003583F583D0E0F09043C0E004F0B420A97D
:10646B009043C2E004F0B4020280030261FF120009
:10647B0096E49043C0F0E49043C1F09043C1E0B484
:05648B000801D3502EB2
:106490001200969043C1E0FB9043C0E075F009A460
:1064A0002488F582E43443F583EB2582F582E435D4
:1064B00083F5837401F09043C1E004F080C89043F9
:1064C000C0E004F0B405BAE490438DF090438EF040
:1064D00090438FF0904392F090439CF090439EF055
:1064E0009043A3F01200937B057A5E794E12590017
:0D64F00012009312F09C7F4812F10F5036FD
:1064FD001200937B057A5E796D125900120093E4B8
:0C650D00FD904275F07F4812F17A5011A9
:106519001200937B057A5E798812590012009380E4
:0A65290018D21A7F44128CEC800F88
:106533001200937B057A5E79991259001200937FBA
:0B6543004812F10F7F9412F10F501A64
:10654E00D236904276E04404F01200937B057A5ED8
:0A655E0079B4125900120093801165
:10656800C2361200937B057A5E79D1125900120067
:08657800937F9C12F10F5046C5
:10658000D237904276E04408F01200937B057A5EA1
:0F65900079EE1259001200937F5412F10F501739
:10659F00D23A904276E04410F07B057A5F79101280
:0765AF005900120093802344
:1065B600C23A7B057A5F793612590012009380132E
:1065C600C237C23A1200937B057A5F795C12590092
:0A65D6001200937F4E12F10F501ACD
:1065E000D23C904276E04420F01200937B057A5F23
:0A65F000797E125900120093801109
:1065FA00C23C1200937B057A5F79A11259001200FE
:0D660A00937F4E12F10F7F9612F10F501A80
:10661700D23B904276E04401F01200937B057A5F0B
:0A66270079C412590012009380118B
:10663100C23B1200937B057A5F79E0125900120088
:08664100937FA512F10F501A1E
:10664900D238904276E04440F01200937B057A5F9D
:0A66590079FC125900120093801121
:10666300C2381200937B057A607916125900120022
:08667300937F9312F10F501305
:10667B00D2391200937B057A6079301259001200DF
:03668B00938011E8
:10668E00C2391200937B057A60794A1259001200C2
:08669E00937F4612F10F501A20
:1066A600D23D904276E04480F01200937B057A60FA
:0A66B600796412590012009380115C
:1066C000C23D1200937B057A60798712590012004F
:1066D000937F4612F10FE4FFFDFB1286E6E4FFFB19
:1066E0007D011286E6E49043C0F09043C0E0B4041C
:1066F00001D34003026774E49043C1F09043C1E0CA
:06670000B40701D350654F
:106706001200969043C1E0FF9043C0E075F009A4E3
:106716002457F582E4344CF583EF2582F582E4357F
:1067260083F583E09043C2F09043C0E0700B904342
:09673600C1E06029E06401602467
:10673F009043C0E0FF9043C1E0FD9043C2E0FB12E5
:10674F0086E69043C0E0FF9043C1E0FD9043C2E076
:10675F00FB1286E69043C1E004F080919043C0E0C5
:0F676F0004F00266EAE49043C0F0E49043C1F006
:10677E001200969043C1E0FB9043C0E02323248493
:10678E00F582E4344CF583EB2582F582E43583F50E
:10679E0083E09043C2F09043C0E07A00C333CA3323
:1067AE00CA2410FF9043C1E0FD9043C2E0FB128962
:1067BE009A9043C0E07A00C333CA33CA2410FF90C4
:1067CE0043C1E0FD9043C2E0FB12899A9043C1E0C1
:1067DE0004F0B4049B9043C0E004F0B4068DE4F0E2
:1067EE009043C0E0249CF582E4344CF583E0FD90A8
:1067FE0043C0E0240AF582E43443F583EDF0904380
:10680E00C0E004F0B406D9904F3AE0FF128CC99064
:10681E004F39E0FF128C85904F38E0FF128C41907B
:10682E004F37E0FF128BFD90429AE0FF128B4D9096
:10683E004F3AE0FF128CC9904F39E0FF128C8590D1
:10684E004F38E0FF128C41904F37E0FF128BFD90D6
:0D685E00429AE0FF128B4D120096303C185C
:09686B007F4E7D7F12F17A500F7F
:106874001200937B057A6079AA1259001200939052
:086884004AFFE0B406004043A6
:10688C00120093904AFFE0FBE4C0E0EBC0E07B0514
:10689C007A6079CB125900158115819043C3744AE3
:1068AC00F0A374FFF0E4FF9043C3E0FCA3E0FD12FF
:0668BC000066EE4F600CC7
:1068C2001200937B057A6079EB12590022904AFFFD
:1068D200E075F010A4FB740A2BF582E4344BF583C7
:1068E200E09043C0F0904AFFE075F010A4FB7409F9
:1068F2002BF582E4344BF583E09043C1F09043C022
:04690200E0B4FF0AF4
:10690600E4F09043C1E004F080069043C0E004F058
:1069160074019043C5F0904AFFE075F010A4FB7433
:106926000A2BFBE4344B9043C3F0A3EBF09043C037
:10693600E0FF9043C3E0FCA3E0FD120066EE4F606B
:1069460005E49043C5F0904AFFE075F010A4FB748F
:10695600092BFBE4344B9043C3F0A3EBF09043C107
:10696600E0FF9043C3E0FCA3E0FD120066EE4F603B
:1069760005E49043C5F0904AFFE075F010A4FB745F
:10698600082BF582E4344BF583E09043C0F0904A3F
:10699600FFE075F010A4FB74072BF582E4344BF589
:0D69A60083E09043C1F09043C0E0B4FF0ACD
:1069B300E4F09043C1E004F080069043C0E004F0AB
:1069C300904AFFE075F010A4FB74082BFBE4344BF2
:1069D3009043C3F0A3EBF09043C0E0FF9043C3E0C8
:1069E300FCA3E0FD120066EE4F6005E49043C5F0A2
:1069F300904AFFE075F010A4FB74072BFBE4344BC3
:106A03009043C3F0A3EBF09043C1E0FF9043C3E096
:106A1300FCA3E0FD120066EE4F6005E49043C5F071
:106A2300904AFFE09043C6F075F010A4FB74072B67
:106A3300F582E4344BF583E0FA904AFFE075F010F9
:106A4300A4FD74082DF582E4344BF583E0FDE42DB9
:106A5300FDE43A9043C3F0A3EDF09043C3E0C0E0FC
:106A6300A3E0C0E0904AFFE02401FFE43400FE7C91
:106A7300277D101254A88EF0D0E0FBD0E0B5F007CC
:0C6A83008FF0EBB5F001D35003026F4719
:106A8F009043C6E004F0904AFFE075F010A4FB7449
:106A9F00052BF582E4344BF583E09043C2F0904A26
:106AAF00FFE075F010A4FB74052BFBE4344B90430F
:106ABF00C3F0A3EBF09043C2E0FF9043C3E0FCA30D
:106ACF00E0FD120066EE4F6005E49043C5F0904A7A
:106ADF00FFE075F010A4FB74062BF582E4344BF540
:106AEF0083E09043C2F0904AFFE075F010A4FB746E
:106AFF00062BFBE4344B9043C3F0A3EBF09043C25F
:106B0F00E0FF9043C3E0FCA3E0FD120066EE4F6090
:106B1F0005E49043C5F0904AFFE075F010A4FB74B4
:106B2F00042BF582E4344BF583E09043C2F0904A96
:106B3F00FFE075F010A4FB74042BFBE4344B90437F
:106B4F00C3F0A3EBF09043C2E0FF9043C3E0FCA37C
:106B5F00E0FD120066EE4F6005E49043C5F0904AE9
:106B6F00FFE075F010A4FB74032BF582E4344BF5B2
:106B7F0083E09043C2F0904AFFE075F010A4FB74DD
:106B8F00032BFBE4344B9043C3F0A3EBF09043C2D1
:106B9F00E0FF9043C3E0FCA3E0FD120066EE4F6000
:106BAF0005E49043C5F0904AFFE075F010A4FB7424
:106BBF00022BF582E4344BF583E09043C2F0904A08
:106BCF00FFE075F010A4FB74022BFBE4344B9043F1
:106BDF00C3F0A3EBF09043C2E0FF9043C3E0FCA3EC
:106BEF00E0FD120066EE4F6005E49043C5F0904A59
:106BFF00FFE075F010A4FB74012BF582E4344BF524
:106C0F0083E09043C2F0904AFFE075F010A4FB744C
:106C1F00012BFBE4344B9043C3F0A3EBF09043C242
:106C2F00E0FF9043C3E0FCA3E0FD120066EE4F606F
:106C3F0005E49043C5F0904AFFE075F010A42400DE
:106C4F00F582E4344BF583E09043C2F0904AFFE0C5
:106C5F0075F010A42400FBE4344B9043C3F0A3EB76
:106C6F00F09043C2E0FF9043C3E0FCA3E0FD1200AD
:106C7F0066EE4F6005E49043C5F0904AFFE075F073
:106C8F0010A4FB74092BF582E4344BF583E0904399
:106C9F00C2F0904AFFE075F010A4FB74092BFBE4DF
:106CAF00344B9043C3F0A3EBF09043C2E0FF90430B
:106CBF00C3E0FCA3E0FD120066EE4F6005E49043D5
:106CCF00C5F0904AFFE075F010A4FB740A2BF58213
:106CDF00E4344BF583E09043C2F0904AFFE075F047
:106CEF0010A4FB740A2BFBE4344B9043C3F0A3EBCB
:106CFF00F09043C2E0FF9043C3E0FCA3E0FD12001D
:106D0F0066EE4F6005E49043C5F0904AFFE075F0E2
:106D1F0010A4FB74072BF582E4344BF583E090430A
:106D2F00C2F0904AFFE075F010A4FB74072BFBE450
:106D3F00344B9043C3F0A3EBF09043C2E0FF90437A
:106D4F00C3E0FCA3E0FD120066EE4F6005E4904344
:106D5F00C5F0904AFFE075F010A4FB74082BF58284
:106D6F00E4344BF583E09043C2F0904AFFE075F0B6
:0D6D7F0010A4FB74082BFBE4344B9043C3BD
:106D8C00F0A3EBF09043C2E0FF9043C3E0FCA3E020
:106D9C00FD120066EE4F6005E49043C5F0904AFF8B
:106DAC00E075F010A4FB740B2BF582E4344BF583E7
:106DBC00E09043C2F0904AFFE075F010A4FB740B16
:106DCC002BFBE4344B9043C3F0A3EBF09043C2E0B5
:106DDC00FF9043C3E0FCA3E0FD120066EE4F60059C
:106DEC00E49043C5F0904AFFE075F010A4FB740CDE
:106DFC002BF582E4344BF583E09043C2F0904AFFCC
:106E0C00E075F010A4FB740C2BFBE4344B9043C3E3
:106E1C00F0A3EBF09043C2E0FF9043C3E0FCA3E08F
:106E2C00FD120066EE4F6005E49043C5F0904AFFFA
:106E3C00E075F010A4FB740D2BF582E4344BF58354
:106E4C00E09043C2F0904AFFE075F010A4FB740D83
:106E5C002BFBE4344B9043C3F0A3EBF09043C2E024
:106E6C00FF9043C3E0FCA3E0FD120066EE4F60050B
:106E7C00E49043C5F0904AFFE075F010A4FB740E4B
:106E8C002BF582E4344BF583E09043C2F0904AFF3B
:106E9C00E075F010A4FB740E2BFBE4344B9043C351
:106EAC00F0A3EBF09043C2E0FF9043C3E0FCA3E0FF
:106EBC00FD120066EE4F6005E49043C5F0904AFF6A
:106ECC00E075F010A4FB740F2BF582E4344BF583C2
:106EDC00E09043C2F0904AFFE075F010A4FB740FF1
:106EEC002BFBE4344B9043C3F0A3EBF09043C2E094
:106EFC00FF9043C3E0FCA3E0FD120066EE4F60057B
:0B6F0C00E49043C5F09043C5E0701115
:106F17001200937B057A617915125900120093804C
:016F27001F4A
:106F28009043C6E0FF7DFF7C4A120066EE4F600F7B
:106F38001200937B057A617943125900120093E598
:106F48008954F044029043C0F0F589758CF1D28CD5
:106F580075D90475F91875E90075EA4075FA407530
:106F6800EB4075FB4075DA4275DB427590FF75D8CA
:106F780040E5D9F0E5D89043C1F0E5F99043C2F077
:106F8800E5E9FBE49043C3F0A3EBF0E5DA9043C5F1
:106F9800F0E5EA9043C6F0759F8275BF0875AF00AB
:106FA80075AA4075BA4075AB4075BB40759A427575
:106FB8009B4275C0FF75E840E59F9043C0F0E5E847
:106FC8009043C1F0E5BF9043C2F0E5AFFBE49043C6
:106FD800C3F0A3EBF0E59A9043C5F0E5AA9043C649
:106FE800F0904D39E020E004C2298002D229904D6A
:096FF80039E020E104C228800BFD
:0E700100D228904C58E0049043C9F0303D284E
:07700F00904D39E020E31170
:107016007F467DFE12F17A50077F16E4FD128FF44B
:017026002247
:107027007F467DFF12F17A50077F16E4FD128FF439
:017037002236
:107038009044D0EBF0A3EAF0A3E9F09044D3EDF04C
:10704800A3ECF0A3E8F09043CAE4F0A3F09044D393
:0C7058001250DD125090FF1200A25038C0
:107064009044D31250DDE004F09044D47003E00463
:10707400F09044D01250E6E004F09044D17003E064
:1070840004F012509012502D9043CBE004F0904342
:10709400CA70BEE004F080B99044D01250DDE4120E
:0B70A40050499043CAE0FEA3E0FF2229
:1070AF009044B7EBF0A3EAF0A3E9F09044BAEDF007
:1070BF00A3ECF0A3E8F09044BDE4F0A3F09044BA41
:0C70CF001250DD125090FF120099503852
:1070DB009044BA1250DDE004F09044BB7003E0041E
:1070EB00F09044B71250E6E004F09044B87003E01F
:1070FB0004F012509012502D9044BEE004F09044D6
:10710B00BD70BEE004F080B99044B71250DDE412BC
:0B711B0050499044BDE0FEA3E0FF22BD
:10712600426567696E6E696E672053656C662D549D
:107136006573740A0020202054657374696E672095
:1071460045787465726E616C205352414D20203033
:1071560078253034582D3078343746460A002020BA
:10716600202020204D656D6F7279206661696C2C38
:107176002041646472657373203078253034580A70
:10718600002020202020202020206265666F726566
:10719600203D203078253032580A0020202020203B
:1071A600202020206D6964202020203D2030782575
:1071B6003032580A0020202020202020202061661E
:1071C60074657220203D203078253032580A002020
:1071D600202020202020202045787465726E616C66
:1071E6002044617461204D656D6F72792028535279
:1071F600414D29205061737365640A0020202020C8
:10720600202020202045787465726E616C204461D0
:107216007461204D656D6F727920285352414D2956
:10722600204661696C65642C20636F6E74696E75A7
:10723600696E670A002069616E6F64655F6D6F6EC7
:107246002025642C2069616E6F64655F6C696D69C9
:107256007420256420210A0020636374726C5F69C0
:107266006E202564210A00206E65775F76616C20AA
:1072760025642C2063757272656E745F76616C206E
:10728600256420210A00696E20636865636B5F6868
:10729600765F755F6C696D69742C20726561645FD9
:1072A600383539312072657475726E656420312007
:1072B600210A00696E20636865636B5F68765F7597
:1072C6005F6C696D69742C20726573756C742069C6
:1072D600732025642C206C696D69742069732025E0
:1072E6006420210A00696E20636865636B5F6876B7
:1072F6005F6C5F6C696D69742C20726561645F38C0
:107306003539312072657475726E656420312021BD
:107316000A00696E20636865636B5F68765F6C5F01
:107326006C696D69742C20726573756C7420697351
:107336002025642C206C696D69742069732025648E
:1073460020210A00436865636B696E672053796E76
:107356006320210A002020207673796E635F636FB5
:10736600756E74203C2033302021200A0020202016
:1073760068667265715F696E203C20333620210A8B
:1073860000436865636B696E6720482053796E63B6
:107396002C2035207365636F6E647320210A0020EC
:1073A600202068667265715F617665726167652027
:1073B6007374696C6C206368616E67696E672021FF
:1073C6000A00436865636B696E672048562C203354
:1073D600207365636F6E647320210A0020202048A5
:1073E60056206C6F7720696E206765745F73796EBF
:1073F600635F706172616D7320210A00202020484E
:1074060056206869676820696E206765745F7379BE
:107416006E635F706172616D7320210A00696E2070
:107426007365745F6461632C20636869705F6E7551
:107436006D207761732025642020210A0020696E63
:10744600207365745F6461632C20676F74206932F2
:1074560063206572726F722C20636869705F6E7547
:107466006D2077617320256420210A00696E2073E0
:1074760065745F64696769706F742C2063686970EE
:107486005F6368616E2069732025642C2069676ECE
:107496006F72656420210A00696E207365745F64EB
:1074A600696769706F742C20636620253032582C0A
:1074B60020636E20253032582C2074656D7020258F
:1074C6003032582C20636320253032582C207661C8
:1074D6006C202530325820210A00696E20736574AD
:1074E6005F64696769706F742C20636869705F6E8A
:1074F600756D2069732025642C2069676E6F72652F
:107506006420210A00696E207365745F6469676987
:10751600706F742C20693263206572726F7220213D
:027526000A0059
:10752800696E207365745F735F6361705F706F72FB
:10753800742C2077726974655F6932635F64617463
:1075480061206661696C656420210A0069326320E4
:107558006661696C65642073657474696E6720641C
:1075680065666C5F656E61626C6520210A00693230
:1075780063206661696C65642073657474696E67FD
:107588002068765F656E61626C6520210A00556E21
:107598006B6E6F776E20436F6E66696720426F6F00
:1075A8007420506172616D657465722027256327A8
:1075B800202530325820210A006765745F73796E80
:1075C800635F706172616D73206661696C656420C8
:1075D800210A00444143204E756D20272564272049
:1075E8006F7574206F662072616E67652020210AAE
:1075F800004441432056616C7565206F7574206F97
:10760800662072616E676520210A00506172616DA3
:10761800657465722076616C7565206F7574206F6E
:10762800662072616E676520210A00556E6B6E6F69
:10763800776E206F7074696F6E20307825303258FD
:10764800202725632720210A00577269746520497D
:10765800324320656570726F6D206661696C732CAA
:1076680020646576696365202530325820210A0038
:10767800577269746520656570726F6D20666169FF
:107688006C656420210A0021200A004C56505320C2
:107698006973206C6F7720210A00566964656F2032
:1076A8002B383056206973206C6F7720210A0048E8
:1076B800565053206973206C6F7720210A00485672
:1076C800505320697320686967682C207368757443
:1076D80074696E6720646F776E20210A00566572A0
:1076E800746963616C206465666C656374696F6E48
:1076F800206F666620210A00486F72697A6F6E747F
:10770800616C206465666C656374696F6E206F6672
:107718006620210A004E69676874206D6F646520D1
:10772800210A00446179206D6F646520210A0048B0
:10773800562053485554444F574E20616374697618
:10774800652C204856206F666620210A004856207E
:1077580053485554444F574E20696E616374697697
:10776800652C204856206F6E20210A00426F6F74E6
:10777800205265636F7264204661696C65642021DC
:107788000A004C4544207772697465206661696C0B
:10779800656420210A006661696C656420777269F6
:1077A80074696E6720566964656F205532313420DC
:1077B800210A004572726F722072656164696E6792
:1077C800204C56505320636F6E74726F6C253031A5
:1077D800642C206465766963652055333125303122
:1077E8006420210A00202B362E3356206C6F772018
:1077F800256420210A00202B3556206C6F77202520
:107808006420210A00202B393056206C6F77202500
:107818006420210A00202D3856206C6F77202564BB
:1078280020210A00202B323456206C6F77202564E3
:1078380020210A00202B313256206C6F77202564D6
:1078480020210A00202D31303056206C6F772025FA
:107858006420210A00202D313256206C6F772025B4
:107868006420210A004572726F7220726561646932
:107878006E6720646576696365202530325820215B
:107888000A00556E6B6E6F776E20636F6D6D616E5B
:107898006420636861722030782530325820210ACC
:1078A80000696E62756670747220307825303258BF
:1078B800202020696E6275666964782030782530EA
:1078C80032582020696E6275666964785F656E64F7
:1078D8002030782530325820210A00556E6B6E6FA3
:1078E800776E206573636170652073657175656E69
:1078F80063652030782530325820272563272021DA
:107908000A00556E6B6E6F776E206D6573736167D5
:1079180065202725642720696E2077726974655F62
:107928006572726F725F6D6573736167655F6E20F4
:03793800210A0021
:10793B00756E657870656374656420636861722029
:10794B00256320210A00257320230A00230A004FF8
:10795B004B20230A004E2F4120230A00426F6F74E5
:10796B00696E672046696E697368656420230A0037
:10797B00426164206D65737361676520696E646530
:10798B007820256420210A0025642C200025642002
:03799B00230A00BC
:10799E00C2231200937B057A7179261259001200C8
:1079AE00937442C0E07474C0E07B057A71793B1227
:1079BE00590015811581D20B90427475450275469A
:1079CE0042754774E546B44706E547B4FF01D34018
:0479DE0003027A9690
:1079E200D20CAB45AA46A947125090F541F4F54492
:1079F200125090F412504912509065446002C20C29
:107A0200AB45AA46A947125090F542125090F41283
:0F7A12005049F543E54165436002C20C200C5713
:107A2100120093C046C0477B057A717964125900F0
:107A310015811581120093E4C0E0C0417B057A7184
:107A4100798712590015811581120093E4C0E0C0B5
:107A5100427B057A7179A1125900158115811200B5
:107A610093E4C0E0C0437B057A7179BB12590015DC
:107A7100811581D223C20B0547E54770040546E510
:107A81004675A61E75A6E10547E54760030279D252
:087A910005460279D2300B0D0D
:0D7A99001200937B057A7179D512590022F5
:0D7AA6001200937B057A72790212590022BA
:0B7AB300904294E004F0B43C00402A34
:0D7ABE00E4F0904295E004F0B43C00401D5F
:0D7ACB00E4F0904296E004F0B41800401082
:107AD800E4F0904298E004F09042977003E004F0DC
:017AE800227B
:037AE90030401218
:107AEC00904F22E090445FF0904F23E0904460F080
:027AFC008010F8
:107AFE00904F20E090445FF0904F21E0904460F072
:097B0E00904F3BE0B55600506CAD
:067B170030332A302E2756
:107B1D00120093904F3BE0FBE4C0E0EBC0E0E4C00B
:107B2D00E0C0557B057A72793B12590074FC2581B2
:107B3D00F581120093C22E904387E075F077A4FB78
:107B4D0024C5F8F582E43442F583E0FA904461F0FF
:107B5D00B40401D3400C904461E024FB904462F0E6
:107B6D008008904461E0904462F0E4FFFD9044622F
:067B7D00E0FB1286E62287
:067B8300302903027CDC46
:107B8900904281E0B55400500F904281E0FAE554EB
:107B9900C39A904463F0800B904281E0C39554905E
:107BA9004463F0904F2EE0F5F0904463E0B5F001A6
:0D7BB900D3500A904281E0904464F0802196
:097BC600E554904464F0303318DA
:107BCF00120093E4C0E0C0547B057A72795E1259BB
:107BDF000015811581120093904387E075F077A40B
:107BEF0024C5F582E43442F583E0904461F090447B
:107BFF0060E0FB90445FE0FFEBC39FF5F0E494007F
:107C0F00904464E0A490445FE025F0904462F0302B
:057C1F003330302E2D72
:107C2400120093904461E0FBE4C0E0EBC0E09044B8
:107C340062E0FBE4C0E0EBC0E07B057A72796D1290
:107C4400590074FC2581F581120093C22E90446181
:0D7C5400E0F5F0904462E0B5F001D350205F
:0E7C61009043C8E0F5F0904462E065F0606486
:107C6F00E4FDFFE0FB1286E6904462E09043C8F02B
:027C7F00805231
:107C8100904461E0FB7A008AF0904462E024FBFDBD
:107C9100E434FFB400078BF0EDB5F001D3400C9054
:107CA1004461E02405904462F08009904461E0045D
:107CB100904462F09043C8E0F5F0904462E065F0D2
:027CC100601051
:107CC300E4FFFDE0FB1286E6904462E09043C8F0D7
:097CD300904464E0904281F0222B
:107CDC00303418904387E075F077A424C5F582E41E
:107CEC003442F583E0904462F08016904387E0754F
:107CFC00F077A42457F582E4344CF583E090446289
:0F7D0C00F09043C8E0F5F0904462E065F060103D
:107D1B00E4FFFDE0FB1286E6904462E09043C8F07E
:017D2B002235
:037D2C00304012D2
:107D2F00904F26E090445FF0904F27E0904460F032
:027D3F008010B2
:107D4100904F24E090445FF0904F25E0904460F024
:067D5100302803027E6DE4
:107D570090427EE0B55300500F90427EE0FAE55323
:107D6700C39A904461F0800B90427EE0C395539094
:107D77004461F0904F2FE0F5F0904461E0B5F001D9
:107D8700D3500A90427EE0904462F08006E553901B
:107D97004462F0904387E075F077A424C5F582E448
:107DA7003442F583A3E0904463F0904460E0FB9095
:107DB700445FE0FFEBC39FFCE49400FEECFF9044BC
:107DC70062E0FD7C001254A890445FE02E9044646A
:107DD700F0904463E0F5F0904464E0B5F001D350CF
:017DE700217A
:0E7DE8009043C9E0F5F0904464E065F0606EF1
:107DF600E4FF7D01E0FB1286E6904464E09043C90F
:037E0600F0805BAE
:107E0900904463E0FB7A008AF0904464E024FBFD2F
:107E1900E434FFB400078BF0EDB5F001D3400C90CA
:107E29004463E02405904464F08009904463E004CD
:107E3900904464F09043C9E0F5F0904464E065F043
:027E49006011C6
:107E4B00E4FF7D01E0FB1286E6904464E09043C9B9
:107E5B00F0904464E090427EF0904462E090427E69
:027E6B00F02203
:107E6D00303419904387E075F077A424C5F582E48A
:107E7D003442F583A3E0904464F08017904387E08B
:107E8D0075F077A42457F582E4344CF583A3E09084
:107E9D004464F09043C9E0F5F0904464E065F0600F
:017EAD0011C3
:107EAE00E4FF7D01E0FB1286E6904464E09043C956
:027EBE00F022B0
:107EC00074FFC39F9043CEF09042CAE09043CFF03E
:107ED00090430DE0FF9043D0F03395E0FE9043CE09
:107EE000E0FD7C001254A8EE9043CCF0A3EFF0909C
:107EF00043CCE0FA9043D0F09043CFE02A9043D0B7
:107F0000F0E4FF7D05E0FB1286E69042C7E0904377
:107F1000CFF090430AE0FF9043D0F03395E0FE901D
:107F200043CEE0FD7C001254A8EE9043CCF0A3EFCA
:107F3000F09043CCE0FA9043D0F09043CFE02A9009
:107F400043D0F0E4FF7D02E0FB1286E69042CBE0F6
:107F50009043CFF090430EE0FF9043D0F03395E094
:107F6000FE9043CEE0FD7C001254A8EE9043CCF08E
:107F7000A3EFF09043CCE0FA9043D0F09043CFE0F1
:107F80002A9043D0F0E4FF7D06E0FB1286E69042A3
:107F9000C8E09043CFF090430BE0FF9043D0F03324
:107FA00095E0FE9043CEE0FD7C001254A8EE904395
:107FB000CCF0A3EFF09043CCE0FA9043D0F09043A4
:107FC000CFE02A9043D0F0E4FF7D03E0FB1286E689
:107FD0009042CCE09043CFF090430FE0FF9043D02D
:107FE000F03395E0FE9043CEE0FD7C001254A8EE05
:107FF0009043CCF0A3EFF09043CCE0FA9043D0F064
:108000009043CFE02A9043D0F0E4FF7D07E0FB12DD
:1080100086E69042C9E09043CFF090430CE0FF9099
:1080200043D0F03395E0FE9043CEE0FD7C00125447
:10803000A8EE9043CCF0A3EFF09043CCE0FA90434D
:10804000D0F09043CFE02A9043D0F0E4FF7D04E0ED
:05805000FB1286E62290
:06805500120096303623F4
:0D805B007F907B027A44795F12F511500A84
:108068007F217D90128FF47F0122904462E0B496C4
:098078000050037F0122E4FF2205
:0E808100120096E49043D5F0203B0302817676
:0D808F007F967B027A4379D112F511500AD9
:10809C007F18E4FD128FF47F01229043D1E0B4905D
:0480AC0001D3400DAF
:1080B0007F1CE0FD128FF474019043D5F09043D201
:0680C000E0B4AF00500D1A
:1080C6007F1BE0FD128FF474019043D5F09043D3EB
:0680D600E0B4AF00500D04
:1080DC007F1DE0FD128FF474019043D5F09043D4D2
:0680EC00E0B4AF00500DEE
:1080F2007F1EE0FD128FF474019043D5F07F987BD0
:0A810200027A4379D112F511500AF8
:10810C007F187D01128FF47F01229043D1E0B4AF30
:03811C0000500D03
:10811F007F19E0FD128FF474019043D5F09043D294
:06812F00E0B4AF00500DAA
:108135007F1AE0FD128FF474019043D5F09043D37C
:07814500E0B4E101D3400D9D
:10814C007F20E0FD128FF474019043D5F09043D45E
:07815C00E0B4E101D3400D86
:108163007F1FE0FD128FF474019043D5F09043D547
:06817300E0FF22E4FF2200
:0681790012009630376E83
:0D817F007F927B027A4379D612F5115012DF
:10818C001200937B057A72798C1259001200937F3E
:10819C0001229043D7E09044B7F09043D6E0F556D7
:1081AC00904F35E0F5F09044B7E0B5F001D3402E98
:1081BC00120093904F35E0FBE4C0E0EBC0E090443C
:1081CC00B7E0FBE4C0E0EBC0E07B057A7279B91252
:1081DC00590074FC2581F5811200937F0122E4FF84
:0481EC0022E4FF2268
:0681F00012009630376D0D
:0D81F6007F927B027A4379DA12F511501264
:108203001200937B057A7279EB1259001200937F67
:1082130001229043DBE09044B7F09043DAE0F55657
:0F822300904F36E0F5F09044B7E0B5F000502EE4
:10823200120093904F36E0FBE4C0E0EBC0E09044C4
:10824200B7E0FBE4C0E0EBC0E07B057A737918127B
:10825200590074FC2581F5811200937F0122E4FF0D
:0482620022E4FF22F1
:06826600120096303723E0
:0D826C007F4D79DE7A437B0212F69C5003B1
:108279007F01229043DEE05404F0B40001D34003AF
:098289007F0122E4FF227F0122A3
:0682920012009630371FB8
:0D8298007F4D79DF7A437B0212F69C500384
:1082A5007F01229043DFE05402F070037F0122E456
:0582B500FF227F012201
:1082BA001200937B057A73794A125900E4FEFDF5A0
:1082CA0049AF527C011254A8EE90427AF0A3EFF023
:1082DA007F01128D1490427AE0FAA3E0FB9043E208
:1082EA00EAF0A3EBF07F01128D14E549B41E0050A9
:0182FA00196A
:1082FB001200937B057A73795B125900120093C2BB
:10830B001A7F11128CEC7F0122AF497E007C01E4B5
:0F831B00FD1254A88E4A8F4BE552B42400501225
:10832A001200937B057A7379731259001200937FB6
:10833A000122E49043E1F0D2097F01128D149042A8
:10834A007AE0FAA3E0FB9043E2EAF0A3EBF0120032
:10835A00937B057A7379871259009043E1E0B4055B
:0C836A000040030284292009030284293A
:10837600904294E09043E0F07F01128D149043E127
:10838600E004F0C2099043E2E0FAF5F0A3E0FB90C6
:10839600427AE0B5F0088BF0A3E0B5F001D34033A4
:1083A60090427AE0FAA3E0FB9043E3E0F8EBC3984F
:1083B600FB9043E2E0F8EA98B40204BB0001D34024
:0183C60012A4
:1083C70090427AE0FAA3E0FB9043E2EAF0A3EBF0F5
:1083D700D2099043E2E0FAF5F0A3E0FB90427AE09D
:1083E700B5F0078BF0A3E0B5F00050309043E2E022
:1083F700FAA3E0FB90427BE0F8EBC398FB90427A4C
:0D840700E0F8EA98B40204BB0001D3400F76
:10841400E0FAA3E0FB9043E2EAF0A3EBF0D2091206
:0884240000960283643009197F
:10842C00C21A7F11128CEC1200937B057A7379A51A
:10843C001259001200937F01221200937B057A736C
:10844C0079C81259007F03128D141281F0EF601954
:10845C00C21A7F88128CEC1200937B057A7379E236
:0F846C001259001200937F0122128179EF6019DB
:10847B00C21A7F88128CEC1200937B057A747902F6
:10848B001259001200937F0122D21A7F11128CEC29
:03849B00E4FF22D9
:06849E002034030285C535
:1084A400E490445FF090445FE0B40401D3400302DD
:1084B400853CE4904460F0904460E0B40701D350FC
:1084C4006E90445FE0B40001D3500A904460E0B47D
:0584D4000101D340523C
:1084D900904460E0FBE4C0E0EBC0E090445FE075ED
:1084E900F009A4FD904387E075F077A424C5F582CF
:1084F900E43442F583ED2582F582E43583F583D0B2
:10850900E02582F582D0E03583F583E0904461F07F
:1085190090445FE0FF904460E0FD904461E0FB120D
:1085290086E6904460E004F0808890445FE004F0BF
:108539000284A9203C030285C4E490445FF090447E
:108549005FE0B40501D35073E4904460F090446057
:07855900E0B40301D3505C04
:10856000904460E0FB90445FE02323FDE4C0E0ED35
:10857000C0E0904387E075F077A424F2F582E434FC
:1085800042F583D0E02582F582D0E03583F583EB98
:108590002582F582E43583F583E0904461F09044D0
:1085A0005FE0C3332410FF904460E0FD904461E03D
:1085B000FB12899A904460E004F0809A90445FE056
:0585C00004F08083229D
:1085C500E490445FF090445FE0B40401D3400302BB
:1085D500865DE4904460F0904460E0B40701D350B8
:1085E5006E90445FE0B40001D3500A904460E0B45B
:0585F5000101D340521A
:1085FA00904460E0FBE4C0E0EBC0E090445FE075CB
:10860A00F009A4FD904387E075F077A42457F5821A
:10861A00E4344CF583ED2582F582E43583F583D085
:10862A00E02582F582D0E03583F583E0904461F05D
:10863A0090445FE0FF904460E0FD904461E0FB12EB
:10864A0086E6904460E004F0808890445FE004F09D
:10865A000285CA203C030286E5E490445FF0904418
:10866A005FE0B40501D35073E4904460F090446035
:07867A00E0B40301D3505CE2
:10868100904460E0FB90445FE02323FDE4C0E0ED13
:10869100C0E0904387E075F077A42484F582E43448
:1086A1004CF583D0E02582F582D0E03583F583EB6C
:1086B1002582F582E43583F583E0904461F09044AE
:1086C1005FE0C3332410FF904460E0FD904461E01B
:1086D100FB12899A904460E004F0809A90445FE034
:0586E10004F08083227B
:1086E6009044E6EFF09044E7EDF09044E8EBF07448
:1086F600019044E9F0EF75F009A42488F582E4348A
:1087060043F583ED2582F582E43583F583E0B401F4
:108716000A9044E8E09044EAF0800D9044E8E0FADC
:1087260074FFC39A9044EAF09044E6E0601B14702C
:10873600030287E314700302883C1470030288BBAB
:098746001470030288EC02891092
:06874F0020360302892E12
:108755009044E7E02400B408005061FA232A90878A
:108765006773028781028789028791028799028749
:0C877500A10287A90287B10287B98040E9
:1087810074039044EBF0803E74099044EBF0803622
:1087910074049044EBF0802E74029044EBF0802638
:1087A10074019044EBF0801E74059044EBF0801648
:1087B10074069044EBF0800E74079044EBF0800651
:1087C100740C9044EBF07F949044EBE0FD9044EA0C
:1087D100E0FB12F231400302892EE49044E9F002F9
:0887E100892E20370302892EC6
:1087E9009044E7E0600B14601014601514601A805F
:0187F900205F
:1087FA0074019044EBF0801E74029044EBF08016F2
:10880A0074039044EBF0800E740B9044EBF08006F6
:10881A00740C9044EBF07F9C9044EBE0FD9044EAAA
:10882A00E0FB12F231400302892EE49044E9F0029F
:08883A00892E20370302892E6C
:108842009044E7E0B403028032500BE060151460FC
:108852001A14601F8045E024FC602814602D146007
:0388620032803829
:1088650074049044EBF0803674059044EBF0802E50
:1088750074069044EBF0802674079044EBF0801E5C
:1088850074089044EBF0801674099044EBF0800E68
:10889500740A9044EBF08006740C9044EBF07F9CD6
:1088A5009044EBE0FD9044EAE0FB12F231507AE4AB
:0988B5009044E9F0807330367044
:0888BE009044E7E0600280082D
:1088C60074089044EBF08006740C9044EBF07F94AF
:1088D6009044EBE0FD9044EAE0FB12F2315049E4AB
:1088E6009044E9F08042303C3F9044E7E0B40C000D
:1088F60050367F9E9044E7E0FD9044E8E0FB12F29C
:10890600315025E49044E9F0801E1200939044E62D
:10891600E0FBE4C0E0EBC0E07B057A7479231259F2
:1089260000158115811200939044E9E070213033DF
:018936001E22
:108937001200939044E6E0FBE4C0E0EBC0E07B0567
:108947007A74794312590015811581120093904466
:10895700E8E0C0E09044E7E0FB9044E6E075F0090A
:10896700A4FDE4C0E0EDC0E0904387E075F077A494
:1089770024C5F582E43442F583D0E02582F582D020
:10898700E03583F583EB2582F582E43583F583D0E3
:03899700E0F022EB
:10899A009044C5EFF09044C6EDF09044C7EBF0E484
:1089AA009044C8F0303C3DEF24F0601224FE60167B
:0E89BA0024FE601A24FE601E24FE6022802629
:1089C800745E9044C8F0801E745C9044C8F08016B1
:1089D800745A9044C8F0800E74589044C8F08006C9
:1089E80074569044C8F0303A109044C5E024E660CC
:0389F800028006F4
:1089FB0074549044C8F03038109044C5E024E460BF
:038A0B00028006E0
:0F8A0E0074529044C8F09044C6E0B40400401F76
:108A1D001200939044C6E0FBE4C0E0EBC0E07B05A0
:108A2D007A74797212590015811581120093229072
:108A3D0044C7E0543F9044C9F09044C5E0540FFB47
:108A4D00E4C313CB13CBEB9044CAF09044C9E0C000
:108A5D00E09044C6E0FBE4C0E0EBC0E09044CAE027
:108A6D002323FD904387E075F077A424F2F582E48B
:108A7D003442F583ED2582F582E43583F583D0E02C
:108A8D002582F582D0E03583F583D0E0F030334C8C
:108A9D001200939044C9E0FBE4C0E0EBC0E09044C9
:108AAD00C6E0FBE4C0E0EBC0E09044CAE0FBE4C0EC
:108ABD00E0EBC0E09044C5E0FBE4C0E0EBC0E0902B
:108ACD004387E0FBE4C0E0EBC0E07B057A74799E60
:108ADD0012590074F62581F5811200939044C8E077
:028AED007022F5
:038AEF0030331E03
:108AF2001200939044C5E0FBE4C0E0EBC0E07B05CC
:108B02007A7479E01259001581158112009322902E
:108B120044C6E0232354FC24A09044CBF09044C7E5
:108B2200E0543F9044C9F09044C8E0FF9044CBE049
:0B8B3200FD9044C9E0FB12F231500F2F
:108B3D001200937B057A75790B125900120093225E
:108B4D009044B7EFF0203701227F4A9044B7E0FD03
:058B5D0012F17A500F37
:108B62001200937B057A757928125900120093221C
:108B72003018047AFE80027AFFEA3030047AF780F5
:108B8200027AFF5A9043C7F0201805C219128BBF10
:038B920020302070
:0C8B95007F4C9043C7E0FD12F17A5010B5
:108BA1001200937B057A75795412590012009322B1
:0E8BB100A218922FA218921A7F22128CEC2288
:108BBF00302F047AFE80027AFFEA3019047AF780A8
:108BCF00027AFF5AFD9043C7F07F4C12F17A501092
:108BDF001200937B057A7579761259001200932251
:0E8BEF00A2199230A219921A7F88128CEC22E1
:108BFD009044B7EFF09044B8744FF0A37437F090F1
:108C0D0044B8E0FCA3E0FD12945F9044B8744CF0BE
:108C1D00A3749DF09044B7E0FF9044B8E0FCA3E04E
:108C2D00FD12945F30380C7F1C7D019044B7E0FB42
:048C3D0012899A22DC
:108C41009044B7EFF09044B8744FF0A37438F090AB
:108C510044B8E0FCA3E0FD12945F9044B8744CF07A
:108C6100A3749EF09044B7E0FF9044B8E0FCA3E009
:108C7100FD12945F30380C7F1C7D029044B7E0FBFD
:048C810012899A2298
:108C85009044B7EFF09044B8744FF0A37439F09066
:108C950044B8E0FCA3E0FD12945F9044B8744CF036
:108CA500A3749CF09044B7E0FF9044B8E0FCA3E0C7
:108CB500FD12945F30380C7F1CE4FD9044B7E0FB57
:048CC50012899A2254
:108CC9009044B7EFF07D3A7C4F12945F3036137FB2
:108CD900909044B7E0FD12F68650077F17E4FD1225
:038CE9008FF422E3
:108CEC00301A08904275E04FF08009EFF4FE904284
:108CFC0075E05EF07F48904275E0FD12F17A500706
:088D0C007F16E4FD128FF42232
:108D14009044B7EFF0E49043E4F09044B7E0F5F00A
:098D24009043E4E0B5F0005015A5
:038D2D002000051E
:108D300012009680F8C200127AB39043E4E004F087
:038D400080DC22B2
:108D43009044BDEFF09044BEEDF09044BFEBF0A330
:108D5300EAF0A3E9F09044BA1250E6ED9044C2F071
:108D6300A3ECF0A3E8F09044B71250DDE41250BB3B
:108D73001250499044BF1250DD125090640A7003A0
:108D8300028E439044BF1250DD125090640D700365
:108D9300028E439044B71250DD1250906480B48029
:108DA3000B09B900010A125090B41E004003028E51
:018DB300437C
:108DB4009044BF1250DD9044C21250E6E004F0909B
:108DC40044C37003E004F012509012502D9044BD3F
:108DD400E0FFC0E09044B71250DD9044BEE0FD09CE
:108DE400B900010A1250902DFD19C0D0B9FF011A23
:108DF400D0D012509034009044BF1250DDE004F003
:108E04009044C07003E004F0125090FF33EFFBD0A5
:078E1400E0FF12F7765002A7
:108E1B00D3229044B71250DD09B900010A125090C9
:108E2B000412504919B9FF011A6003028D761250D2
:108E3B009004125049028D769044C21250DDE41218
:108E4B0050499044BDE0FF9044B71250DD9044BEB2
:108E5B00E0FD09B900010A1250902DFD19C0D0B9DF
:0F8E6B00FF011AD0D0125090E4FB12F77650029C
:048E7A00D322C3221A
:108E7E009044B7EEF0A3EFF09044B9EBF0A3EAF014
:108E8E00A3E9F09044BCEDF0A3ECF0A3E8F090441D
:108E9E00B91250DD125090640A607B9044B91250A2
:108EAE00DD125090640D606E9044BC1250DD125075
:108EBE00906480B4800B09B900010A125090B41F5F
:038ECE00005053FE
:108ED1009044B91250DDE004F09044BA7003E0040C
:108EE100F0125090FF9044B7E0FCA3E0FDE004F0E5
:0E8EF1009044B77003E004F012945FEF60024B
:108EFF00D3229044BC1250DD09B900010A125090E0
:108F0F000412504919B9FF011A70821250900412BD
:108F1F005049028E9CE4FF9044B7E0FCA3E0FD12A1
:058F2F00945FEF6002F9
:108F3400D3229044BC1250DDE02402F09044BDE002
:058F44003400F0C3221F
:108F4900E5309043E5F0E5329043E6F09043E5E003
:0C8F5900F5F09043E6E0B5F001D34006CF
:108F6500E490417EF0229043E5E0FAF5F09043E687
:108F7500E0B5F001D34024E4C0E07403C0E07B0217
:108F85007A41797E9043E5E02400FDE43440FCED30
:0B8F9500F87D0212557915811581222C
:108FA0009043E5E0FB7480C39BFBE49400C0E0EBDE
:108FB000C0E07B027A41797EE02400FDE43440FC8D
:108FC000EDF87D0212557915811581E4C0E0740237
:108FD000C0E09043E5E0FA7480C39A247EFBE43459
:108FE00041FAEBF97B027D027C407800125579153D
:048FF0008115812244
:108FF4009044CCEFF09044CDEDF01200939044CC2B
:10900400E024FFB42300400302938CFA232A9090B7
:1090140016730290820290A90290B50290D0029039
:10902400DC0290E802910F02912A02938C0291369D
:1090340002914202914E02915A0291660291720289
:10904400917E02918A0291960291A20291AE0291BE
:10905400BA0291C60291D20291DE029207029222D2
:1090640002923D02925802927302928E0292A902D7
:0E90740092C40292DF0292FA02936602938C7B
:109082009044CDE0FBE4C0E0EBC0E0E0FD3395E0CE
:10909200C0E0EDC0E07B057A75799612590074FC48
:1090A2002581F5810293A47B057A7579C112590055
:1090B2000293A49044CDE0FBE4C0E0EBC0E07B056A
:1090C2007A7579DB125900158115810293A47B050B
:1090D2007A7579F91259000293A47B057A7679138D
:1090E2001259000293A49044CDE0FD3395E0C0E014
:1090F200EDC0E0E0FBE4C0E0EBC0E07B057A76790E
:109102003312590074FC2581F5810293A49044CD59
:10911200E0FBE4C0E0EBC0E07B057A7679511259BE
:1091220000158115810293A47B057A76797812590C
:10913200000293A47B057A76798F1259000293A4D8
:109142007B057A7679931259000293A47B057A768D
:1091520079A21259000293A47B057A7679B7125943
:10916200000293A47B057A7679C61259000293A471
:109172007B057A7679E51259000293A47B057A770A
:1091820079001259000293A47B057A77791D12594E
:10919200000293A47B057A77792B1259000293A4DB
:1091A2007B057A7779371259000293A47B057A7787
:1091B20079551259000293A47B057A777974125972
:1091C200000293A47B057A77798A1259000293A44C
:1091D2007B057A77799E1259000293A49044CDE0E0
:1091E200FBE4C0E0EBC0E0E02401FBE43400C0E0BB
:1091F200EBC0E07B057A7779BB12590074FC2581BC
:10920200F5810293A49044CDE0FBE4C0E0EBC0E022
:109212007B057A7779ED125900158115810293A4A5
:109222009044CDE0FBE4C0E0EBC0E07B057A7779C7
:10923200FE125900158115810293A49044CDE0FBE2
:10924200E4C0E0EBC0E07B057A78790D1259001595
:109252008115810293A49044CDE0FBE4C0E0EBC011
:10926200E07B057A78791D125900158115810293E8
:10927200A49044CDE0FBE4C0E0EBC0E07B057A784B
:10928200792C125900158115810293A49044CDE0E6
:10929200FBE4C0E0EBC0E07B057A78793C12590030
:1092A200158115810293A49044CDE0FBE4C0E0EB6C
:0692B200C0E07B057A78A4
:1092B800794C125900158115810293A49044CDE090
:1092C800FBE4C0E0EBC0E07B057A78795D125900D9
:1092D800158115810293A49044CDE0FBE4C0E0EB36
:1092E800C0E07B057A78796D1259001581158102E5
:1092F80093A49044CDE0FBE4C0E0EBC0E07B057AAA
:1093080078798A125900158115811200939043B714
:10931800E0FBE4C0E0EBC0E09043B6E0FBE4C0E073
:10932800EBC0E09043B5E0FBE4C0E0EBC0E07B05B8
:109338007A7879A912590074FA2581F58112009377
:10934800E4C0E0C032C0E0C031C0E0C0307B057A84
:109358007879A912590074FA2581F581803E9044E4
:10936800CDE0FD3395E0C0E0EDC0E0E0FBE4C0E017
:10937800EBC0E07B057A7879E312590074FC25810B
:10938800F58180189044CCE0FBE4C0E0EBC0E07BC2
:10939800057A79790A1259001581158112009322EC
:1093A8009044B7EFF01200939044B7E0FB3395E098
:1093B800C0E0EBC0E07B057A79793B125900158152
:0693C80015811200932242
:1093CE009044D6EBF0A3EAF0A3E9F0120093904498
:1093DE00D6E0C0E0A3E0C0E0A3E0C0E07B057A7970
:0F93EE00795112590074FD2581F58112009322E7
:1093FD009044B7EFF01200939044B7E014600B1453
:0A940D00601314601B146023802C10
:109417007B057A79795712590080397B057A7979F2
:109427005A125900802E7B057A797960125900808B
:10943700237B057A79796712590080189044B7E041
:10944700FBE4C0E0EBC0E07B057A79797B12590039
:0894570015811581120093221A
:10945F00904440EFF0904441ECF0A3EDF012006621
:04946F00EE4F600A52
:0D9473007F08E4FD128FF47F0122E4FF2248
:10948000E53105312400F582E43440F583740DF0B4
:10949000E4FE7F0D12006CE531B480004003E4F57A
:1094A00031E53105312400F582E43440F583E4F000
:1094B000E531B480004003E4F531853132E4FE7FCC
:0794C0000A12006CD2042225
:1094C700120093E49043E7F09043E7E0240AF58223
:1094D700E43443F583E0FB3395E0C0E0EBC0E07B89
:1094E700057A797993125900158115819043E7E040
:1094F70004F0B405D390430FE0FB3395E0C0E0EBF5
:10950700C0E07B057A797998125900158115811287
:039517000093229C
:10951A00646576696365206E6F7420617661696C33
:08952A0061626C6520210A005A
:1095320041646472203D203078253034580A00237B
:109542000A0042616E6B206F7574206F6620726133
:109552006E676520696E20426F6F7420746F2046BB
:109562006C6173682C2064697361626C656420218C
:109572000A00556E6B6E6F776E20626F6F74206299
:109582006C6F636B210A0042616420636F6E6669CF
:1095920067206E756D62657220210A00210A004300
:1095A2006F6E666967204E756D6265722025642351
:1095B2000A00446163204E616D6520256320697352
:1095C200206E6F74207265636F676E697A656421BD
:1095D2000A004F4B230A00696E20636463632C20E8
:1095E200636F6E6669675F6E756D206973206F7554
:1095F20074206F662072616E6765282076616C2028
:109602003D2025642920210A0044616320436861CA
:109612006E6E656C202564206973206F7574206FEF
:10962200662072616E67652C206461635F6E756D82
:1096320020697320256420210A00556E6B6E6F77B6
:109642006E204856204F7074696F6E202D2025635E
:1096520020210A004D6F64656C204E756D62657243
:10966200203D200025630020230A002700272069CF
:109672006E76616C69642C2069203D20256420216E
:109682000A00256420686F757273206973203E207A
:109692007468616E2032332C2069676E6F72656464
:1096A20020210A002564206D696E75746573206936
:1096B20073203E207468616E2035392C2069676EF4
:1096C2006F72656420210A002564207365636F6EE2
:1096D2006473206973203E207468616E2035392CD2
:1096E2002069676E6F72656420210A00636F6E667F
:1096F2006967206F7065726174696E672074696D45
:10970200653A20756E6B6E6F776E206F7074696F3D
:109712006E20256320210A0020756E6578706563CE
:1097220074656420646967697420256320210A00D6
:10973200777269746520656570726F6D2066616904
:109742006C656420210A004C696D6974203D2025F6
:109752006420230A0053657269616C204E756D6244
:109762006572203D2000253033752C253033752C51
:10977200253033752C253033752C253033752C2547
:109782003033752C253033750A00566964656F5F76
:109792002B38305620253033750A00416E6F6465D0
:1097A2002043757272656E7420253033752C20410A
:1097B2006E6F646520566F6C746167652025303367
:1097C200750A00466F63757320566F6C7461676526
:1097D20020253033752C20473220566F6C74616718
:1097E2006520253033750A002D3856202530337513
:1097F2002C202B39305620253033752C202B323437
:109802005620253033752C202B313256202530330B
:10981200750A002B362E335620253033752C202B1B
:10982200355620253033752C202D313256202530E7
:1098320033752C202D3130305620253033750A00F7
:109842004164647220307825303458203D203078CD
:10985200253032580A006175746F20626F6F742070
:10986200656E61626C656420230A006175746F2005
:10987200626F6F742064697361626C656420230A8D
:1098820000436F6E666967204E756D6265722025B2
:10989200640A00436F6E666967204E616D65203D04
:1098A20020000A002531642C2531642C25730A001E
:1098B200556E6B6E6F776E20444143206E616D650D
:1098C20020210A00253033752C0025303375002CF9
:1098D2002530337520230A002530337520230A00F2
:1098E200446163204E616D65202563206973207594
:1098F2006E7265636F676E697A656420210A00691A
:109902006E2064642E2C20636620253032582C2071
:10991200646E20253032582C2074656D70202530FD
:10992200325820210A00556E6B6E6F776E204461AB
:109932006320537065636966696572202563202020
:03994200210A00F7
:10994500562532642E2530326420230A0025642CE6
:109955002000256420230A00485620557070657242
:10996500204C696D6974203D2025640A0048562005
:109975004C6F776572204C696D6974203D202564B4
:109985000A00416E6F64652043757272656E7420BE
:109995004C696D6974203D2025640A0048562043B2
:1099A5006F6E74726F6C2056616C7565203D202555
:1099B500642C202564200A00466F63757320436F6D
:1099C5006E74726F6C2056616C7565203D20256440
:1099D5002C202564200A00473220436F6E74726F75
:1099E5006C2056616C7565203D2025642C2025640E
:1099F500200A00566964656F202B38305620436F66
:109A05006E74726F6C2056616C7565203D202564FF
:109A15002C20256420230A004C4544203D20307825
:109A25002530325820230A006661696C656420215F
:109A35000A00004E2F4100312C00302C0031200A45
:109A45000030200A004C696D6974732025642C254B
:109A5500642C25642C25642C25642C25642C256414
:109A65002C25642C25642C2564200A0042432030D3
:109A75002C00424320312C00300A00310A004E6987
:109A8500676874204D6F646520230A00446179205E
:109A95004D6F646520230A00253034642C2530324F
:109AA500642C253032642C253032640A0025640A82
:109AB500005573657220436F6E74726F6C7320442A
:109AC500697361626C656420230A005573657220B1
:109AD500436F6E74726F6C7320456E61626C656462
:109AE50020230A005673796E632046726571756589
:109AF5006E6379203D202532642E2530326420485E
:109B05007A20200A004873796E6320467265717564
:109B1500656E6379203D202532642E253032642020
:109B2500487A2020230A004D6F64656C20547970B3
:109B350065203D20256420230A0043617061626928
:109B45006C697479203D20256420230A00556E69CF
:109B550074204E756D626572203D2000556E6B6EEA
:109B65006F776E20646973706C617920636F6D6DBA
:109B7500616E64207175616C696669657220256323
:109B8500202530325820210A0009256420210A00A9
:109B9500486F72697A6F6E74616C2053697A6520BB
:109BA500256420210A00486F72697A6F6E74616CB2
:109BB5002043656E74657220256420210A00693290
:109BC50063207772697465206661696C210A007586
:109BD5006E6B6E6F776E206C20636F6D6D616E645A
:109BE500202725632720210A0044657669636520BF
:109BF500307825303258204F4B20230A004E432021
:109C05004465766963652030782530325820230A0B
:109C1500004E5220446576696365203078253032E0
:109C25005820230A00556E6B6E6F776E2070696E33
:109C350067206F7074696F6E20210A0048532025D4
:109C450030336420202048432025303364200A0027
:109C550056532025303364202020564320253033A9
:109C650064200A00566572746963616C2053697AD1
:109C75006520256420210A00566572746963616C4C
:109C85002043656E74657220256420210A00240A2C
:109C9500004853202D20486F72697A6F6E74616C8D
:109CA5002053697A652020202020204843202D203C
:109CB500486F72697A6F6E74616C2043656E746566
:109CC500720A005653202D20566572746963616CC3
:109CD5002053697A6520202020202020205643200B
:109CE5002D20566572746963616C2043656E7465D9
:109CF500720A0052554E4E494E472C205A20464F67
:109D050052204D454E552C203F20464F522056415E
:109D15004C5545532020230A004350552053687560
:109D250074646F776E0A00256320697320616E2065
:109D3500756E6B6E6F776E207265736574207479BE
:109D450070652C20646973706C6179206973207368
:089D5500746F707065640A0070
:109D5D00904465EBF0A3EAF0A3E9F0125090FF12E6
:109D6D00009950139044651250DD120087EE904219
:079D7D002FF0A3EFF080625C
:109D84009044651250DD125090FF1200A890446573
:109D94001250E6EF12502D12506524D5600E24FEA9
:0C9DA400601A24EC602624F4602E803647
:109DB000904230E004F090422F702BE004F08026B7
:109DC000904230E024FFF090422FE034FFF0801604
:109DD00090422F74FFF0A374F0F0800A90422F7429
:109DE0004DF0A37439F012009390422FE0C0E0A32D
:109DF000E0C0E07B057A9579321259001581158112
:109E00001200937B057A957941125900E4FE7F0197
:019E1000222F
:109E1100904465EBF0A3EAF0A3E9F0C2051250907B
:109E2100FF1200A89044651250DDEF125049125004
:0F9E31009024BB603814606224F36003029EE942
:109E4000120090D20D9042017440F0A3E4F09042D1
:109E5000037447F0A374FFF0D2051200937B057AD8
:109E6000957941125900E4FE7F0122029EFF120003
:109E700090D20E9042017448F0A3E4F09042037433
:109E80004FF0A374FFF0D2051200937B057A957909
:109E900041125900E4FE7F01228064904467E0048F
:109EA000F09044667003E004F09044651250DD12B7
:109EB000008AEB904465F0A3EAF0A3E9F0904465D2
:0A9EC0001250DD125090643360165A
:109ECA001200937B057A9579441259001200931275
:109EDA000090E4FEFF22D207E4FE7F0122801612E0
:109EEA0000937B057A957974125900120093120037
:0A9EFA0090E4FEFF22E4FE7F012247
:109F0400904465EBF0A3EAF0A3E9F0125090FF123D
:109F140000A89044651250DDEF125049125090B4DD
:109F24004F0302B3885041125090B4460302ABE58C
:109F3400501C12509024BF606E14700302A05E1473
:109F4400700302A0EC14700302A4A302C3391250DC
:109F54009024B9700302AD3F14700302AD7924FB61
:109F6400700302AF3D02C339125090B4550302C1CD
:109F7400EB501A12509024B0700302B8D924FD702B
:109F84000302BD9D14700302C19802C3391250909C
:109F940024AA700302C1F514700302C25924FD708F
:079FA4000302C2E302C3390E
:109FAB00120093904467E004F09044667003E00461
:109FBB00F09044651250DD12008AEB904465F0A3DB
:109FCB00EAF0A3E9F09044651250DD125090FF12B5
:0E9FDB0000A8EF9043ECF0E024BD6002805738
:109FE900904467E004F09044667003E004F0904404
:109FF900651250DD12008AEB904465F0A3EAF0A3E4
:10A00900E9F09044651250DD1250909043ECF0B4A1
:02A01900300E07
:09A01B007F4E7DFF12F17A501A0C
:05A02400E4FE7F0122B3
:07A029009043ECE0B4311F8D
:09A030007F4E7D7F12F17A50167B
:10A03900E4FE7F0122800F7F069043ECE0FD128F42
:10A04900F4E4FE7F01227B057A95794112590012C9
:10A05900009302C34D904467E004F0904466700396
:10A06900E004F09044651250DD12008AEB904465DB
:10A07900F0A3EAF0A3E9F09043E8744AF0A374FE70
:10A08900F09044651250DD12509024D060051460A0
:03A099001C8034F4
:10A09C0074AAFF904468F09043E8E0FCA3E0FD1242
:10A0AC00945FEF6033E4FE7F0122E4FF904468F09C
:10A0BC009043E8E0FCA3E0FD120066EE4F6019E46B
:10A0CC00FE7F01227F019044651250DD125090FDFD
:10A0DC00128FF4E4FE7F01227F021293FD02C34D26
:10A0EC00904467E004F09044667003E004F0904400
:10A0FC00651250DD12008AEB904465F0A3EAF0A3E0
:10A10C00E9F09044651250DD125090FF1200A8EF58
:10A11C009043ECF0E0B4350302A3ED5023E024D0DF
:10A12C00700302A3ED14700302A3ED14700302A3D9
:10A13C00ED14700302A3ED14700302A3ED02A498B6
:10A14C00E024BF601B24FD605D14700302A23A245E
:10A15C00F7700302A2C424FB700302A3A802A49804
:04A16C00E5BA600BE5
:10A170007F02E4FD128FF4E4FEFF22904387E07536
:10A18000F077A4249BF582E43442F583E4F0A3F055
:10A19000904387E075F077A4249DF582E43442F57E
:10A1A00083E4F0A3F07F011293FDE4FE7F0122021D
:10A1B000C34D904467E004F09044667003E004F0FF
:10A1C0009044651250DD12008AEB904465F0A3EADA
:10A1D000F0A3E9F09044651250DD1250909043ECEA
:10A1E000F01200939043ECE06480B4B000403790EC
:0BA1F00043ECE06480B4B501D3502BB9
:10A1FB009043ECE0FB3395E0FAEB24D0FBEA34FF21
:10A20B00EB904469F075F077A42499F582E434421D
:10A21B00F583E4F07F011293FD80097B057A957934
:10A22B0089125900120093E4FE7F012202C34D9064
:10A23B004467E004F09044667003E004F0904465DA
:10A24B001250DD12008AEB904465F0A3EAF0A3E90B
:10A25B00F09044651250DD1250909043ECF01200D8
:10A26B00939043ECE06480B4B000403C9043ECE04E
:08A27B006480B4B501D350303A
:10A283009043ECE0FB3395E0FAEB24D0FBEA34FF98
:10A29300EB904469F075F077A42499F582E4344295
:10A2A300F5837401F07B057A957941125900800991
:10A2B3007B057A957989125900E4FE7F012202C356
:10A2C3004D904467E004F09044667003E004F0901E
:10A2D30044651250DD12008AEB904465F0A3EAF066
:10A2E300A3E9F090446AE4F0A3F09044651250DDD2
:10A2F3001250909043ECF09043ECE0640D606AE000
:10A30300640A606590446AE06480B48005A3E0B4A5
:04A313001E00505583
:10A317009043ECE0FE90446AE0FCA3E0FD904387A5
:10A32700E075F077A424A5F582E43442F583ED25A2
:10A3370082F582EC3583F583EEF0904467E004F014
:10A347009044667003E004F09044651250DD1250AB
:10A35700909043ECF090446BE004F090446A709363
:10A36700E004F0808E90446AE0FCA3E0FD90438710
:10A37700E075F077A424A5F582E43442F583ED2552
:10A3870082F582EC3583F583E4F01200937B057A3E
:10A39700957941125900120093E4FE7F012202C30E
:07A3A7004D1282BAEF6016AF
:10A3AE001200937B057A95799E12590090446AE4C7
:10A3BE00F0A3F002C34D90446AE4F0A304F012003F
:10A3CE0093904387E0FBE4C0E0EBC0E07B057A9519
:10A3DE0079A11259001581158112009302C34D9077
:10A3EE0043ECE0FB3395E0FAEB24D0FBEA34FFEBD1
:10A3FE00904387F090446AE4F0A3F090446CE4F04C
:02A40E00A3F0B9
:10A4100090446CE0FEA3E0FF90446BE075F009A46B
:10A42000FB904387E075F077A424C5F582E43442BD
:10A43000F583EB2582F582E43583F583EF2582F5FC
:10A4400082EE3583F583E0904468F090446BE0FF42
:10A4500090446DE0FD904468E0FB1286E690446D08
:10A46000E004F0B408AA90446BE004F0B4059A90BC
:10A470004387E075F077A4249AF582E43442F583AB
:10A48000E0FF904468F0128B4D1200937B057A95A3
:10A49000794112590002C34D9043ECE0FF1293A89A
:10A4A00002C34D904467E004F09044667003E004FA
:10A4B000F09044651250DD12008AEB904465F0A3E1
:10A4C000EAF0A3E9F09044651250DD125090FF12BB
:10A4D0000099500C9044651250E6125065FE8011B0
:10A4E0009044651250E6125065FF1200A8EF33EF5A
:0CA4F000FEEE9043ECF0FF120099502C9F
:10A4FC009043ECE0FB3395E0FAEB24D0FBEA34FF1D
:0EA50C00FAEB90446EF0BB0500500302A675FA
:10A51A007F0390446EE0FD128FF4E4FEFF22904325
:0BA52A00ECE0FF12009F400302A6546B
:10A535009043ECE0B4480302A5DF5022E0B44402A6
:10A54500806B500EE024BF603B14604614605102DE
:10A55500A633E024BB606524FE607002A633E024C8
:10A56500B7700302A5EE24FE700302A5FC14700368
:10A5750002A60A24F9700302A61724FD700302A699
:04A585002502A633D2
:10A58900740490446EF00490446FF002A67574034D
:10A5990090446EF01490446FF002A67574FF9044D5
:10A5A9006EF090446FF002A675741090446EF074CA
:10A5B9000490446FF002A675741290446EF074040E
:10A5C90090446FF002A675741490446EF074049070
:10A5D900446FF002A675740190446EF074049044BF
:10A5E9006FF002A675741690446EF0740490446F6F
:10A5F900F08079741890446EF0740490446FF08080
:10A609006BE490446EF0740890446FF0805E741AA5
:10A6190090446EF0740490446FF08050740290443A
:10A629006EF0740790446FF080421200939043ECEF
:10A63900E0FB3395E0C0E0EBC0E07B057A9579B4A7
:0BA6490012590015811581E4FEFF226C
:10A654001200939043ECE0FB3395E0C0E0EBC0E0E4
:10A664007B057A9579B412590015811581E4FEFFB2
:10A6740022904467E004F09044667003E004F09094
:10A6840044651250DD12008AEB904465F0A3EAF0B1
:10A69400A3E9F09044651250DD125090FF12009926
:10A6A400500C9044651250E6125065FB80139044A0
:10A6B400651250E6125065FF1200A8EF3395E0EFE3
:0EA6C400FBEB9043ECF0BB5002800302A97147
:0CA6D20090446EE0B40F00400302A78823
:10A6DE00E4904470F0904470E0F5F090446FE0B573
:08A6EE00F001D3500302A84F54
:10A6F600904470E0FB90446EE075F009A4FDE4C060
:10A70600E0EDC0E0904387E075F077A4FF24C5F53F
:10A7160082E43442F583D0E02582F582D0E03583A9
:10A72600F583EB2582F582E43583F583E090446872
:10A73600F0904470E0FB90446EE075F009A4FDEFE4
:10A746002457F582E4344CF583ED2582F582E43511
:10A7560083F583EB2582FBE435839043E8F0A3EB96
:10A76600F0904468E0FF9043E8E0FCA3E0FD12941B
:10A776005FEF6005E4FE7F0122904470E004F00282
:02A78600A6E348
:10A78800E4904470F0904470E0F5F090446FE0B5C8
:08A79800F001D3500302A84FA9
:10A7A000904470E0FBE4C0E0EBC0E090446EE05405
:10A7B0000FFDE4C313CD13CDED232354FCFFE4C000
:10A7C000E0EFC0E0904387E075F077A424F2F582D3
:10A7D000E43442F583D0E02582F582D0E03583F57C
:10A7E00083D0E02582F582D0E03583F583E0904484
:10A7F00068F0904470E0FBED232354FCFFE4C0E0DC
:10A80000EFC0E0904387E075F077A42484F582E4FC
:10A81000344CF583D0E02582F582D0E03583F58392
:10A82000EB2582FBE435839043E8F0A3EBF0904402
:10A8300068E0FF9043E8E0FCA3E0FD12945FEF6066
:10A8400005E4FE7F0122904470E004F002A78DE44D
:09A85000904470F0E4904469F0BA
:10A85900904469E0FB904470E075F077A4FD24A56D
:10A86900F582E43442F583EB2582F582E43583F5FC
:10A8790083E0904468F0904469E0FBED2437F58269
:10A88900E4344CF583EB2582FBE435839043E8F00F
:10A89900A3EBF0904468E0FF9043E8E0FCA3E0FDFF
:10A8A90012945FEF6005E4FE7F0122904470E07529
:10A8B900F077A42499F582E43442F583E090446862
:10A8C900F0904470E075F077A4FB742B2BFBE43413
:10A8D9004C9043E8F0A3EBF0904468E0FF9043E824
:10A8E900E0FCA3E0FD12945FEF6005E4FE7F012226
:10A8F900904469E004F0B42002800302A85990440E
:10A9090070E004F0B40202800302A85490446EE09F
:03A91900B4014541
:10A91C00904387E075F077A4249AF582E43442F5ED
:10A92C0083E0904468F0904387E075F077A4FB7463
:10A93C002C2BFBE4344C9043E8F0A3EBF0904468F0
:10A94C00E0FF9043E8E0FCA3E0FD12945FEF6005AC
:10A95C00E4FE7F01221200937B057A9579D412597B
:10A96C0000E4FEFF229043ECE0B44302800302AA11
:01A97C001DBD
:10A97D00904387E0B401004078904387E0B4020033
:02A98D00506F09
:0AA98F00E4904469F0E4904470F095
:10A99900904470E0FB904469E075F009A424C5F582
:10A9A90082E43442F583EB2582F582E43583F5832D
:10A9B900E0904468F0904469E0FF904470E0FD90B5
:10A9C9004468E0FB1286E6904470E004F0B408C0E5
:10A9D900904469E004F0B405B290429AE0FF9044D3
:10A9E90068F0128B4D1200937B057A9579D4125930
:10A9F90000E4FEFF22120093904387E0FBE4C0E0ED
:10AA0900EBC0E07B057A9579D9125900158115813A
:10AA1900E4FEFF229044651250DD125090FF1200AF
:03AA2900995065DC
:10AA2C009044651250DD125090FD3395E0FCED24FE
:10AA3C00D0FDEC34FFED904471F090446FE0F5F0F4
:10AA4C00904471E0B5F001D3403B90446EE0B4010A
:09AA5C0008904471E06408602CCC
:10AA650012009390446EE0FBE4C0E0EBC0E090443C
:10AA750071E0FBE4C0E0EBC0E07B057A96790B1250
:10AA8500590074FC2581F581E4FEFF22904467E0BE
:10AA950004F09044667003E004F09044651250DDC4
:10AAA50012008AEB904465F0A3EAF0A3E9F0740282
:10AAB500904492F0A37444F0A37472F090449212FF
:10AAC50050DD9044651250E61270AFEE90446AF086
:10AAD500A3EFF09044921250DD120087EE9044955A
:10AAE500F0A3EFF0904495E06480B48002A3E040C9
:10AAF50011904495E06480B48006A3E0B4FF01D3CF
:02AB0500400B03
:10AB07007F04E4FD128FF4E4FFFE229044651250A7
:10AB1700E690446BE028FA90446AE03CFC90446578
:10AB2700EDF0A3ECF0A3EAF0904467E004F0904462
:10AB3700667003E004F09044651250DD12008AEB62
:10AB4700904465F0A3EAF0A3E9F090446EE0B40105
:08AB570043904471E0B4083C96
:10AB5F00904495E06480B48006A3E0B43F01D340F5
:10AB6F0009904495E4F0A3743FF0904496E0FF12EF
:10AB7F008B4D904496E0FC904387E075F077A424CA
:0CAB8F009AF582E43442F583ECF0803B40
:10AB9B0090446EE0B40901D3401D90446EE0B41FA5
:03ABAB0000501443
:10ABAE0090446EE0FF904471E0FD904496E0FB12FD
:04ABBE00899A8012DE
:10ABC20090446EE0FF904471E0FD904496E0FB12E9
:10ABD20086E6D2341200937B057A9579D412590015
:10ABE20002C34D904467E004F09044667003E004B1
:10ABF200F09044651250DD12008AEB904465F0A398
:10AC0200EAF0A3E9F09044651250DDE004F09044CC
:10AC1200667003E004F0125090FF1200A8EF904318
:10AC2200ECF0E0B433028039500EE024D060181406
:10AC3200601D14602302ACD0E024CC602C1460317F
:07AC420024E5603502ACD0EF
:10AC4900E49043EEF002ACDF74019043EEF002AC05
:10AC5900DF74029043EEF002ACDF74039043EEF030
:10AC6900807474049043EEF0806C74059043EEF0A8
:09AC7900806490446AE4F0A3F049
:10AC820090446AE0FAA3E0240AF582EA3443F583A9
:10AC9200E09043EDF090446AE0FAA3E0249CFBEAE2
:10ACA200344C90422FF0A3EBF09043EDE0FF904242
:10ACB2002FE0FCA3E0FD12945F90446BE004F0B43B
:10ACC20006BE7F021293FDE4FE7F0122800F7F0603
:10ACD2009043ECE0FD128FF4E4FE7F012212009318
:10ACE2009044651250DD120087EE9043EAF0A3EF24
:10ACF200F09043EAE06480B48006A3E0B4FF01D39D
:02AD0200502AD5
:10AD04009043EBE02480FB9043EAE034FFEB904374
:10AD1400EDF09043EEE0240AF582E43443F583EB4E
:0AAD2400F07F011293FDE4FEFF2210
:10AD2E007F05E4FD128FF4120093E4FFFE2202C3AE
:08AD3E004D90446AE4F0A3F01B
:07AD460090446CE4F0A3F05F
:10AD4D00D2C5C2C590446DE004F0B464F390446B79
:10AD5D00E004F090446A7003E004F0E0B413DAA369
:10AD6D00E0B488D57F011293FD02C34D904467E096
:10AD7D0004F09044667003E004F09044651250DDD9
:10AD8D0012008AEB904465F0A3EAF0A3E9F0904439
:10AD9D00651250DD125090FF1200A8EF9043ECF0B9
:10ADAD00904467E004F09044667003E004F0904432
:10ADBD00651250DD12008AEB904465F0A3EAF0A312
:10ADCD00E9F09044651250DD125090FF1200995039
:01ADDD005223
:10ADDE007402904492F0A37444F0A37472F0904401
:10ADEE00921250DD9044651250E61270AFEE904410
:10ADFE006AF0A3EFF09044921250DD120087EE90AD
:10AE0E004495F0A3EFF0904495E06480B48006A3DF
:07AE1E00E0B4FF01D3400B7B
:10AE25007F05E4FD128FF4E4FEFF229043ECE0B4CD
:10AE35004C0280605015E024BF602524FB607E1421
:10AE4500700302AED114606602AF16E024AE700343
:10AE550002AEEF24FD602314700302AEE002AF16CC
:10AE6500904496E0FF7D3B7C4F12945FEF600302B8
:10AE7500AF377F011293FD02AF37904496E0FF7D17
:10AE8500357C4F12945FEF600302AF377F01129359
:10AE9500FD02AF37904496E0FF7D367C4F12945FFC
:10AEA500EF600302AF377F011293FD02AF37904485
:10AEB50096E0FF128BFD7F021293FD8075904496FC
:10AEC500E0FF128C417F021293FD8066904496E06C
:10AED500FF128C857F021293FD8057904496E0FF08
:10AEE500128CC97F021293FD80489043BAE0FF128D
:10AEF5008BFD9043BCE0FF128C419043BBE0FF12F9
:10AF05008C859043B9E0FF128CC97F021293FD80B6
:10AF1500219043ECE0FB3395E0C0E0EBC0E07B051E
:10AF25007A96793C12590015811581120093E4FE39
:10AF3500FF2212009302C34D904467E004F0904451
:10AF4500667003E004F09044651250DD12008AEB50
:10AF5500904465F0A3EAF0A3E9F09044651250DD52
:10AF6500E004F09044667003E004F0125090FF1284
:10AF750000A8EF3395E0EF9043ECF090446AE4F0DD
:10AF8500A3F09043ECE0B44C0302B1135021E0244C
:10AF9500BD604014700302B01F24FE700302B0664A
:10AFA50014700302B09914700302B0E002B26BE0B2
:10AFB50024B0700302B15A24FD700302B18D1470E0
:10AFC5000302B1C014700302B1F314700302B22579
:03AFD50002B26B5A
:03AFD800303C37D3
:10AFDB0074029044B7F0A37444F0A3746AF0740243
:10AFEB009044BAF0A37444F0A37497F07FAE7D2025
:0BAFFB009044651250DD128D4350168B
:0CB006007F077DAE128FF4E4FE7F012274
:10B012007F031293FDE4FE7F012202B27D303737B7
:10B0220074029044B7F0A37444F0A3746AF07402FB
:10B032009044BAF0A37444F0A37497F07FAA7D20E1
:0BB042009044651250DD128D43501643
:0CB04D007F077DAA128FF4E4FE7F012231
:10B059007F031293FDE4FE7F012202B27D7E4E7FC3
:10B069001A9044651250DD786A7C447D02128E7E06
:02B07900500C79
:10B07B007F08E4FD128FF4E4FE7F01227B027A4409
:10B08B0079977D027C4E781A1255BC02B27D30380E
:01B09B00377D
:10B09C0074029044B7F0A37444F0A3746AF0740281
:10B0AC009044BAF0A37444F0A37497F07FA47D206D
:0BB0BC009044651250DD128D435016C9
:0CB0C7007F077DA4128FF4E4FE7F0122BD
:10B0D3007F031293FDE4FE7F012202B27D7E4D7F4A
:10B0E300BA9044651250DD786A7C447D02128E7EEC
:02B0F300500CFF
:10B0F5007F08E4FD128FF4E4FE7F01227B027A448F
:10B1050079977D027C4D78BA1255BC02B27D303BF1
:01B115003702
:10B1160074029044B7F0A37444F0A3746AF0740206
:10B126009044BAF0A37444F0A37497F07FA87D20EE
:0BB136009044651250DD128D4350164E
:0CB141007F077DA8128FF4E4FE7F01223E
:10B14D007F031293FDE4FE7F012202B27D7E4D7FCF
:10B15D009A9044651250DD786A7C447D02128E7E91
:02B16D00500C84
:10B16F007F08E4FD128FF4E4FE7F01227B027A4414
:10B17F0079977D027C4D789A1255BC02B27D7E4D37
:10B18F007F199044651250DD786A7C447D02128EDF
:03B19F007E500CD3
:10B1A2007F08E4FD128FF4E4FE7F01227B027A44E1
:10B1B20079977D027C4D78191255BC02B27D7E4E84
:10B1C2007FBA9044651250DD786A7C447D02128E0B
:03B1D2007E500CA0
:10B1D5007F08E4FD128FF4E4FE7F01227B027A44AE
:10B1E50079977D027C4E78BA1255BC02B27D7E4DB0
:10B1F5007F5A9044651250DD786A7C447D02128E38
:03B205007E500C6C
:10B208007F08E4FD128FF4E4FE7F01227B027A447A
:10B2180079977D027C4D785A1255BC805830363764
:10B2280074029044B7F0A37444F0A3746AF07402F3
:10B238009044BAF0A37444F0A37497F07FAC7D20D7
:0BB248009044651250DD128D4350163B
:0CB253007F077DAC128FF4E4FE7F012227
:10B25F007F031293FDE4FE7F012280127F0690434D
:10B26F00ECE0FB33EBFD128FF4E4FE7F012274025E
:10B27F00904492F0A37444F0A37497F01200937B60
:10B28F00057A96795612590090446AE06480B4802A
:10B29F0006A3E0B40001D3407390446AE06480B425
:09B2AF008005A3E0B42000506307
:10B2B80090446AE4F0A3F0904497E09043ECF09057
:0AB2C80043ECE0640A603EE0603BE6
:10B2D200E0FB3395E0C0E0EBC0E07B057A9679664F
:10B2E2001259001581158190446BE004F090446A74
:10B2F2007003E004F0A3E02497FA90446AE0344437
:10B30200F5838A82E09043ECF080BA7B057A9679E5
:09B31200691259001200938067D2
:10B31B007B057A96796D1259009044921250DD128A
:10B32B005090640A60379044921250DD1250906036
:10B33B002C9044921250DDE004F09044937003E0A3
:10B34B0004F0125090FD3395E0C0E0EDC0E07B05BA
:10B35B007A9679661259001581158180BC90446AE2
:10B36B00E0C0E0A3E0C0E07B057A96796F1259004C
:10B37B001581158112009312009302C34D904467FF
:10B38B00E004F09044667003E004F09044651250C2
:10B39B00DD12008AEB904465F0A3EAF0A3E9F0908C
:10B3AB0044651250DDE004F09044667003E004F055
:10B3BB00125090FF1200A8EF9043ECF0E0B453034F
:10B3CB0002B5845023E024BD700302B5F714603B33
:10B3DB0024FC700302B49E24FB700302B51124FD00
:10B3EB00700302B68102B8B9E024AA700302B72534
:10B3FB0014700302B77714700302B7C914700302F9
:0BB40B00B81B14700302B86A02B8B945
:10B416009044651250DD120087EE9043E8F0A3EFEA
:10B42600F09043E8E0904469F09043E9E09044707E
:10B43600F0120093904AFFE075F010A42400FBE49C
:10B44600344B9043E8F0A3EBF0904469E0FF90435F
:0CB45600E8E0FCA3E0FD12945FEF60034F
:10B4620002C34D904AFFE075F010A4FB74012BFB60
:10B47200E4344B9043E8F0A3EBF0904470E0FF908B
:10B4820043E8E0FCA3E0FD12945FEF600302B8D64C
:10B492007B057A95794112590002C34D9044651299
:10B4A20050DD120087EE9043E8F0A3EFF012009314
:0FB4B2009043E8E0B40006A3E0B41701D3400FC5
:0FB4C1007B057A96798412590012009302B8D64F
:10B4D0009043E9E0904469F0904AFFE075F010A4D1
:10B4E000FB74022BFBE4344B9043E8F0A3EBF090A9
:10B4F0004469E0FF9043E8E0FCA3E0FD12945FEFB5
:10B50000600302B8D67B057A95794112590002C3CF
:10B510004D9044651250DD120087EE9043E8F0A391
:10B52000EFF01200939043E8E0B40006A3E0B43BD0
:04B5300001D3400FF4
:0FB534007B057A9679A612590012009302B8D6B9
:10B543009043E9E0904469F0904AFFE075F010A45D
:10B55300FB74032BFBE4344B9043E8F0A3EBF09034
:10B563004469E0FF9043E8E0FCA3E0FD12945FEF41
:10B57300600302B8D67B057A95794112590002C35C
:10B583004D9044651250DD120087EE9043E8F0A31E
:10B59300EFF01200939043E8E0B40006A3E0B43B5D
:04B5A30001D3400F81
:0FB5A7007B057A9679CA12590012009302B8D622
:10B5B6009043E9E0904469F0904AFFE075F010A4EA
:10B5C600FB74042BFBE4344B9043E8F0A3EBF090C0
:10B5D6004469E0FF9043E8E0FCA3E0FD12945FEFCE
:10B5E600600302B8D67B057A95794112590002C3E9
:10B5F6004D9044651250DD120087EE9043E8F0A3AB
:10B60600EFF09043E8E0904469F09043E9E090441D
:10B6160070F0120093904AFFE075F010A4FB7405D9
:10B626002BFBE4344B9043E8F0A3EBF0904469E045
:10B63600FF9043E8E0FCA3E0FD12945FEF60030295
:10B64600C34D904AFFE075F010A4FB74062BFBE493
:10B65600344B9043E8F0A3EBF0904470E0FF904346
:10B66600E8E0FCA3E0FD12945FEF600302B8D67B2E
:10B67600057A95794112590002C34D9044651250DE
:10B68600DD120087EE9043E8F0A3EFF09043E8E088
:10B69600904469F09043E9E0904470F01200939072
:10B6A6004AFFE075F010A4FB74092BFBE4344B90C1
:10B6B60043E8F0A3EBF0904469E0FF9043E8E0FC38
:10B6C600A3E0FD12945FEF600302C34D904469E06E
:10B6D600FC904AFFE075F010A4FB74092BF582E498
:10B6E600344BF583ECF0904AFFE075F010A4FB7440
:10B6F6000A2BFBE4344B9043E8F0A3EBF090447044
:10B70600E0FF9043E8E0FCA3E0FD12945FEF6003E6
:10B7160002B8D67B057A95794112590002C34D903D
:10B7260044651250DD120087EE9043E8F0A3EFF077
:10B73600EF904469F0120093904AFFE075F010A470
:10B74600FB740B2BFBE4344B9043E8F0A3EBF09037
:10B756004469E0FF9043E8E0FCA3E0FD12945FEF4C
:10B76600600302B8D67B057A95794112590002C367
:10B776004D9044651250DD120087EE9043E8F0A329
:10B78600EFF0EF904469F0120093904AFFE075F0F5
:10B7960010A4FB740C2BFBE4344B9043E8F0A3EBB2
:10B7A600F0904469E0FF9043E8E0FCA3E0FD1294CA
:10B7B6005FEF600302B8D67B057A9579411259008E
:10B7C60002C34D9044651250DD120087EE9043E8A7
:10B7D600F0A3EFF0EF904469F0120093904AFFE077
:10B7E60075F010A4FB740D2BFBE4344B9043E8F08A
:10B7F600A3EBF0904469E0FF9043E8E0FCA3E0FD92
:10B8060012945FEF600302B8D67B057A95794112F0
:02B816005900D7
:10B8180002C34D9044651250DD120087EE9043E854
:10B82800F0A3EFF0EF904469F0120093904AFFE024
:10B8380075F010A4FB740E2BFBE4344B9043E8F036
:10B84800A3EBF0904469E0FF9043E8E0FCA3E0FD3F
:10B8580012945FEF70787B057A957941125900024E
:10B86800C34D9044651250DD120087EE9043E8F016
:10B87800A3EFF0EF904469F0120093904AFFE0754F
:10B88800F010A4FB740F2BFBE4344B9043E8F0A3B7
:10B89800EBF0904469E0FF9043E8E0FCA3E0FD1280
:10B8A800945FEF70297B057A95794112590002C39C
:10B8B8004D1200939043ECE0FB3395E0C0E0EBC001
:10B8C800E07B057A9679EE1259001581158102C33D
:10B8D8004D904467E004F09044667003E004F090F3
:10B8E80044651250DD12008AEB904465F0A3EAF03B
:10B8F800A3E9F09044651250DD125090FF1200A8A1
:10B90800EF9043ECF0E0B4430302BA15500FE02483
:10B91800D0602314603B24EF605202BD87E024B856
:10B92800700302BAB624FC700302BBAB24FE70039A
:06B9380002BD0102BD8703
:10B93E00D228D22990446AE4F0A304F01200937B3B
:10B94E00057A95794112590002C34DC228C2299039
:10B95E00446AE4F0A304F01200937B057A957941D2
:10B96E0012590002C34D904467E004F09044667093
:10B97E0003E004F09044651250DD12008AEB90440F
:10B98E0065F0A3EAF0A3E9F09044651250DD125081
:0AB99E0090FF120099400302BD9AC9
:10B9A8009044651250DD1250909043ECF0E024D0A2
:07B9B800600514601B8032E2
:10B9BF00D22890446AE4F0A304F01200937B057A36
:10B9CF0095794112590002BD9AC22890446AE4F059
:10B9DF00A304F01200937B057A9579411259000266
:10B9EF00BD9A1200939043ECE0FB3395E0C0E0EB7F
:10B9FF00C0E07B057A97791A1259001581158112CB
:10BA0F000093E4FEFF22904467E004F090446670D8
:10BA1F0003E004F09044651250DD12008AEB90446D
:10BA2F0065F0A3EAF0A3E9F09044651250DD1250DF
:0ABA3F0090FF120099400302BD9A27
:10BA49009044651250DD1250909043ECF0E024D000
:07BA5900600514601B803240
:10BA6000D22990446AE4F0A304F01200937B057A93
:10BA700095794112590002BD9AC22990446AE4F0B6
:10BA8000A304F01200937B057A95794112590002C4
:10BA9000BD9A1200939043ECE0FB3395E0C0E0EBDD
:10BAA000C0E07B057A97791A125900158115811229
:10BAB0000093E4FEFF22904467E004F09044667037
:10BAC00003E004F09044651250DD12008AEB9044CC
:10BAD00065F0A3EAF0A3E9F09044651250DD12503E
:10BAE00090FF1200A8EF9043ECF0904467E004F060
:10BAF0009044667003E004F09044651250DD12003B
:10BB00008AEB904465F0A3EAF0A3E9F09044651253
:0BBB100050DD125090FF120099507D94
:10BB1B009044651250DD120087EF904468F090431B
:0BBB2B00ECE024BE600514600E8018E2
:10BB360090422F744FF0A3742FF0801F90422F7401
:10BB46004FF0A3742EF080131200937B057A95793B
:10BB56009E125900120093E4FEFF22904468E0FF13
:0FBB660090422FE0FCA3E0FD120066EE4F60104E
:10BB75001200937B057A977932125900E4FEFF2271
:10BB85001200937B057A957941125900120093E4CE
:03BB9500FEFF228E
:10BB98001200937B057A95799E125900120093E45E
:10BBA800FEFF22904467E004F09044667003E004CE
:10BBB800F09044651250DD12008AEB904465F0A3C2
:10BBC800EAF0A3E9F09044651250DD125090FF129C
:07BBD8000099400302BCE1EB
:10BBDF009044651250DD125090FB9043ECF033957A
:10BBEF00E0FAEB24D0FBEA34FF90446AF0A3EBF0C9
:10BBFF0090446AE0FAA3E0FBEABA0002800302BCB9
:10BC0F0092EB2400B40800507AFA232A90BC1F73D9
:10BC1F0002BC3902BC3902BC3902BC3902BC650214
:0ABC2F00BC6502BC6502BC658059CB
:10BC3900904387E075F077A424C5F582E43442F592
:10BC490083E0904468F090446BE02420FB90446AC0
:10BC5900E0344F90422FF0A3EBF0803E904387E011
:10BC690075F077A424C5F582E43442F583A3E09006
:10BC79004468F090446BE02420FB90446AE0344F20
:10BC890090422FF0A3EBF080117F069043ECE0FB8C
:10BC990033EBFD128FF4E4FEFF22904468E0FF903D
:0DBCA900422FE0FCA3E0FD12945FEF600B62
:10BCB6007F0AE4FD128FF4E4FEFF22120093904403
:10BCC60068E0FBE4C0E0EBC0E07B057A97794912B7
:0BBCD6005900158115811200938011A8
:10BCE1007F069043ECE0FB33EBFD128FF4E4FEFFA3
:10BCF1002290446AE4F0A304F0FF1293FD02C34DC5
:10BD0100904467E004F09044667003E004F09044CE
:10BD1100651250DD12008AEB904465F0A3EAF0A3AE
:10BD2100E9F09044651250DD125090FF12009950D5
:01BD310068A9
:10BD32009044651250DD1250909043ECF0E024D014
:0DBD4200600B14600C14600D146010801470
:10BD4F00D22A8047C22A8043D22AC240803DD22ABB
:10BD5F00D24080371200939043ECE0FB3395E0C064
:10BD6F00E0EBC0E07B057A97791A1259001581151F
:10BD7F0081120093E4FEFF221200937B057A9579DE
:10BD8F009E12590090446AE4F0A3F002C34D904410
:10BD9F0067E004F09044667003E004F0904465128D
:10BDAF0050DD12008AEB904465F0A3EAF0A3E9F0AE
:10BDBF009044651250DDE004F09044667003E00497
:10BDCF00F0125090FF1200A8EF3395E0EF9043EC84
:10BDDF00F090446AE4F0A3F09043ECE0B44C03021B
:10BDEF00BF6B501EE024BD603814607C24FE7003CE
:10BDFF0002BEBE14700302BEF114700302BF3802FC
:10BE0F00C08DE024B0700302BFB224FD700302BFE7
:10BE1F00E514700302C01724FE700302C04902C06C
:01BE2F008D85
:03BE3000303C376C
:10BE330074029044B7F0A37444F0A3746AF07402DC
:10BE43009044BAF0A37444F0A37497F07FAEE4FD7A
:0BBE53009044651250DD128D43501624
:0CBE5E007F077DAE128FF4E4FE7F01220E
:10BE6A007F031293FDE4FE7F012202C08D30373733
:10BE7A0074029044B7F0A37444F0A3746AF0740295
:10BE8A009044BAF0A37444F0A37497F07FAAE4FD37
:0BBE9A009044651250DD128D435016DD
:0CBEA5007F077DAA128FF4E4FE7F0122CB
:10BEB1007F031293FDE4FE7F012202C08D7E4E7F3F
:10BEC1003A9044651250DD786A7C447D02128E7E80
:02BED100500C13
:10BED3007F08E4FD128FF4E4FE7F01227B027A44A3
:10BEE30079977D027C4E783A1255BC02C08D30386A
:01BEF3003717
:10BEF40074029044B7F0A37444F0A3746AF074021B
:10BF04009044BAF0A37444F0A37497F07FA4E4FDC2
:0BBF14009044651250DD128D43501662
:0CBF1F007F077DA4128FF4E4FE7F012256
:10BF2B007F031293FDE4FE7F012202C08D7E4D7FC5
:10BF3B00DA9044651250DD786A7C447D02128E7E65
:02BF4B00500C98
:10BF4D007F08E4FD128FF4E4FE7F01227B027A4428
:10BF5D0079977D027C4D78DA1255BC02C08D303B4D
:01BF6D00379C
:10BF6E0074029044B7F0A37444F0A3746AF07402A0
:10BF7E009044BAF0A37444F0A37497F07FA8E4FD44
:0BBF8E009044651250DD128D435016E8
:0CBF99007F077DA8128FF4E4FE7F0122D8
:10BFA5007F031293FDE4FE7F012202C08D7E4D7F4B
:10BFB5007A9044651250DD786A7C447D02128E7E4B
:02BFC500500C1E
:10BFC7007F08E4FD128FF4E4FE7F01227B027A44AE
:10BFD70079977D027C4D787A1255BC02C08D7E4DD3
:10BFE7007F3A9044651250DD786A7C447D02128E58
:03BFF7007E500C6D
:10BFFA007F08E4FD128FF4E4FE7F01227B027A447B
:10C00A0079977D027C4D783A1255BC80767E4E7FB8
:10C01A00DA9044651250DD786A7C447D02128E7E85
:02C02A00500CB8
:10C02C007F08E4FD128FF4E4FE7F01227B027A4448
:10C03C0079977D027C4E78DA1255BC8044303637C5
:10C04C0074029044B7F0A37444F0A3746AF07402C1
:10C05C009044BAF0A37444F0A37497F07FACE4FD61
:0BC06C009044651250DD128D43501609
:0CC077007F077DAC128FF4E4FE7F0122F5
:10C083007F031293FDE4FE7F01227402904492F039
:10C09300A37444F0A37497F07B057A9779571259E8
:10C0A3000012009390446AE06480B48006A3E0B475
:10C0B3000001D3407390446AE06480B48005A3E038
:05C0C300B420005063F1
:10C0C80090446AE4F0A3F0904497E09043ECF09039
:0AC0D80043ECE0640A603EE0603BC8
:10C0E200E0FB3395E0C0E0EBC0E07B057A96796631
:10C0F2001259001581158190446BE004F090446A56
:10C102007003E004F0A3E02497FA90446AE0344418
:10C11200F5838A82E09043ECF080BA7B057A9679C7
:09C12200691259001200938067B4
:10C12B007B057A96796D1259009044921250DD126C
:10C13B005090640A60379044921250DD1250906018
:10C14B002C9044921250DDE004F09044937003E085
:10C15B0004F0125090FD3395E0C0E0EDC0E07B059C
:10C16B007A9679661259001581158180BC90446AC4
:10C17B00E0C0E0A3E0C0E07B057A96796F1259002E
:10C18B001581158112009312009302C34D904467E1
:10C19B00E004F09044667003E004F09044651250A4
:10C1AB00DD12008AEB904465F0A3EAF0A3E9F0906E
:10C1BB0044651250DD125090FF1200A8EF9043EC33
:0EC1CB00F0E024D0600814600914600A800AB5
:10C1D900C2268006D2268002D2267F011293FD0252
:10C1E900C34DC2257F011293FD02C34D904467E000
:10C1F90004F09044667003E004F09044651250DD49
:10C2090012008AEB904465F0A3EAF0A3E9F09044A8
:10C21900651250DD125090FF1200A8EF9043ECF028
:10C22900E024D0600B14600E14600F1460108014A9
:10C23900C225C2338012D225800ED233800AD2257C
:10C24900D2338004C225C2337F011293FD02C34D4C
:10C25900904467E004F09044667003E004F0904471
:10C26900651250DD12008AEB904465F0A3EAF0A351
:10C27900E9F09044651250DD120087EE9043E8F032
:0EC28900A3EFF09043E8E0B40102A3E0503AC6
:0FC297009043E9E0FF7D397C4D12945F303D36D6
:07C2A6009043E9E020E312E0
:10C2AD007F467DFE12F17A50197F16E4FD128FF450
:02C2BD00801DE2
:10C2BF007F467DFF12F17A50147F16E4FD128FF442
:02C2CF00800BE2
:10C2D1007F05E4FD128FF4E4FEFF227F011293FD3E
:10C2E100806A904467E004F09044667003E004F0D3
:10C2F1009044651250DD12008AEB904465F0A3EA88
:10C30100F0A3E9F09044651250DD125090FF120045
:10C31100A8EF9043ECF0E024D06005146008800A97
:10C32100C23ED2348004D23ED2341200937B057ACD
:10C3310095794112590080147F069044651250DDB1
:10C34100125090FD33128FF4E4FEFF22E4FE7F01D0
:01C3510022C9
:10C35200904410EBF0A3EAF0A3E9F0904413E4F068
:10C36200A3F012008AEB904410F0A3EAF0A3E9F0E4
:10C372009044101250DD125090FF1200A890441009
:10C382001250E6EF12502D12506524BFB41900402E
:10C392000302E055FA232A90C39D7302C3EB02C540
:10C3A2008B02C66102C72C02D30A02D35502E055A2
:10C3B20002D4CF02E05502E05502E05502D5EE026A
:10C3C200D62802D8B902E05502D92F02E05502E080
:10C3D2005502DA4E02DCD402DE5C02DE8402DEE8C2
:09C3E20002DF1102DF3A02E0550E
:10C3EB00120093E4C0E0C059C0E0C058C0E0C05791
:10C3FB00C0E0C055C0E0C054C0E0C053C0E0C05264
:10C40B007B057A97796812590074F22581F58112B0
:05C41B000093303634EF
:0DC420007F907B027A4379EF12F511500CEA
:10C42D007F217D90128FF4E4FE7F01229043F2E094
:10C43D00FBE4C0E0EBC0E07B057A97798C125900E4
:0AC44D001581158112009330396942
:0DC457007F927B027A4379EF12F511500CB1
:10C464007F217D92128FF4E4FE7F01229043F0E05D
:10C47400FBE4C0E0EBC0E09043EFE0FBE4C0E0EBA2
:10C48400C0E07B057A97799D12590074FC2581F5EB
:10C49400811200939043F1E0FBE4C0E0EBC0E09034
:10C4A40043F2E0FBE4C0E0EBC0E07B057A9779C59A
:10C4B40012590074FC2581F581120093203B03027C
:02C4C400C5743D
:0DC4C6007F967B027A4379EF12F511500C3E
:10C4D3007F217D96128FF4E4FE7F01229043F2E0E8
:10C4E300FBE4C0E0EBC0E09043F1E0FBE4C0E0EB31
:10C4F300C0E09043F0E0FBE4C0E0EBC0E09043EF2A
:10C50300E0FBE4C0E0EBC0E07B057A9779EA1259DF
:10C513000074F82581F5811200937F987B027A439A
:07C5230079EF12F511500C35
:10C52A007F217D98128FF4E4FE7F01229043F2E08E
:10C53A00FBE4C0E0EBC0E09043F1E0FBE4C0E0EBD9
:10C54A00C0E09043F0E0FBE4C0E0EBC0E09043EFD2
:10C55A00E0FBE4C0E0EBC0E07B057A98791512595C
:10C56A000074F82581F5811200937B057A9579414B
:10C57A00125900120093904413E4F0A304F002E06D
:10C58A009090422F74FFF0A374F0F090422FE0FADB
:10C59A00A3E0F99044157402F0A3EAF0A3E9F0903D
:06C5AA004413E4F0A3F0CD
:10C5B0001200939044151250DD125090FDE4C0E03B
:10C5C000EDC0E090422FE0C0E0A3E0C0E07B057A40
:10C5D00098794212590074FC2581F581904230E02F
:10C5E00004F090422F7003E004F0904417E004F050
:10C5F0009044167003E004F0904414E004F0B40892
:10C60000AF120093904AFEE0FBE4C0E0EBC0E074A0
:10C610004AC0E074FEC0E07B057A98794212590066
:10C6200074FC2581F58112009390FFF0E0B4AA0814
:10C6300090FFF1E06455600790FFF2E0B43413908E
:10C640004AFEE064AA600B7B057A9879581259007B
:10C6500080097B057A98796D12590012009302E0E7
:10C6600090120093904387E0FBE4C0E0EBC0E07BD6
:10C67000057A987983125900158115811200937BF0
:10C68000057A987995125900904413E4F0A3F0903C
:10C690004413E0FCA3E0FD904387E075F077A42409
:10C6A000A5F582E43442F583ED2582F582EC3583ED
:0DC6B000F583E0904418F0904418E0604CD1
:10C6BD00E0FB3395E0C0E0EBC0E07B057A96796650
:10C6CD0012590015811581904414E004F090441323
:10C6DD007003E004F0E0FCA3E0FD904387E075F00B
:10C6ED0077A424A5F582E43442F583ED2582F58205
:10C6FD00EC3583F583E0904418F080AE7B057A9895
:10C70D0079A41259001200937B057A95794112593B
:10C71D0000120093904413E4F0A304F002E0909013
:10C72D004412E004F09044117003E004F0904410C2
:10C73D001250DD12008AEB904410F0A3EAF0A3E949
:10C74D00F09044101250DD125090FF1200A8EF33FC
:10C75D00EF904418F09044101250DD125090FF12DB
:07C76D00009F400302D2D23D
:10C77400904418E0B4490302C816502EE0B44502B0
:10C7840080725012E024BF604E14700302C851241A
:10C79400FE605202D0A4E024BA700302CC561460A6
:10C7A4006214700302C85F02D0A4E0B4500302C84C
:10C7B4007D5015E024B5606914700302C84324FE5B
:10C7C400700302D03302D0A4E024AD606324FD7072
:07C7D4000302C86E02D0A4AD
:10C7DB007404904419F00490441AF002D0CD7410F4
:10C7EB00904419F0740490441AF002D0CD74129056
:10C7FB004419F0740490441AF002D0CD7414904490
:10C80B0019F0740490441AF002D0CD7416904419A8
:10C81B00F0740490441AF002D0CD7418904419F0BF
:10C82B00740490441AF002D0CD741A904419F07429
:10C83B000490441AF002D0CDE4904419F07408909F
:10C84B00441AF002D0CD7403904419F01490441A9A
:10C85B00F002D0CD7401904419F0740490441AF096
:10C86B0002D0CD7402904419F0740790441AF00270
:10C87B00D0CD904412E004F09044117003E004F02A
:10C88B009044101250DD12008AEB904410F0A3EA92
:10C89B00F0A3E9F09044101250DD125090FF1200FB
:10C8AB00A8EF33EF904418F012009F400302CC40E6
:10C8BB00904418E0B4490302C9475028E0B445023C
:10C8CB00805C5012E024BF603814700302C98224CC
:10C8DB00FE603C02CA20E024B9605214700302C906
:10C8EB009002CA20E024B5606214607D24FE7003C0
:10C8FB0002C9AE24FB606324FD700302C99F02CA08
:01C90B00200B
:10C90C007404904419F00490441AF002CA33741061
:10C91C00904419F0740490441AF002CA33741290C3
:10C92C004419F0740490441AF002CA3374149044FD
:10C93C0019F0740490441AF002CA33741690441916
:10C94C00F0740490441AF002CA337418904419F02D
:10C95C00740490441AF002CA33741A904419F07497
:10C96C000490441AF002CA33E4904419F07408900D
:10C97C00441AF002CA337403904419F01490441A08
:10C98C00F002CA337401904419F0740490441AF004
:10C99C0002CA337402904419F0740790441AF002DE
:09C9AC00CA33904413E4F0A3F037
:10C9B500120093904414E075F077A4FB2437F582B8
:10C9C500E4344CF5837402C0E0E583C0E0E582C041
:10C9D500E0EB242BF582E4344CF583E0FBE4C0E086
:10C9E500EBC0E0904413E0C0E0A3E0C0E07B057A33
:10C9F5009879A612590074F92581F581904414E0BF
:10CA050004F0B402AB1200937B057A957941125973
:10CA150000120093E4FE7F012280131200937B0530
:10CA25007A9879B2125900120093E4FEFF229044DD
:0ACA350019E0B40F00400302CB53D8
:10CA3F00120093E490441BF090441AE024FEFBE4B0
:10CA4F0034FFFAF5F090441BE0FDE4B5F0078BF0EE
:10CA5F00EDB5F001D35055E0FBE4C0E0EBC0E09042
:10CA6F004419E075F009A4FD904387E075F077A4B1
:10CA7F002457F582E4344CF583ED2582F582E435B5
:10CA8F0083F583D0E02582F582D0E03583F583E00E
:10CA9F00FDE4C0E0EDC0E07B057A9879C61259003D
:10CAAF001581158190441BE004F0808C90441AE0AE
:10CABF00FB904419E075F009A4FDE4C0E0EDC0E07F
:10CACF00904387E075F077A42457F582E4344CF552
:10CADF0083D0E02582F582D0E03583F583E582248B
:10CAEF00FFFFE58334FFFEEB2FF582E43EF583E095
:10CAFF00FBE4C0E0EBC0E07B057A9879CC125900DB
:0BCB0F0015811581904419E0B4012845
:10CB1A00904387E075F077A4242CF582E4344CF531
:10CB2A0083E0FBE4C0E0EBC0E07B057A9879D112A0
:10CB3A0059001581158180097B057A967969125900
:09CB4A0000120093E4FE7F0122B9
:10CB5300120093904419E0540FFBE4C313CB13CB9F
:10CB6300EB90441CF0904413E4F0A3F090441AE0DB
:10CB730024FEFBE434FFFAF5F0904413E0B5F0082B
:10CB83008BF0A3E0B5F001D3505D904413E0C0E017
:10CB9300A3E0C0E090441CE02323FB904387E075AF
:10CBA300F077A42484F582E4344CF583EB2582F5F5
:10CBB30082E43583F583D0E02582F582D0E03583A6
:10CBC300F583E0FDE4C0E0EDC0E07B057A9879C62B
:10CBD30012590015811581904414E004F090441318
:10CBE300708AE004F0808590441AE0FB90441CE0D6
:10CBF3002323FD904387E075F077A42484F582E432
:10CC0300344CF583ED2582F582E43583F583E582A3
:10CC130024FFFDE58334FFFCEB2DF582E43CF58333
:10CC2300E0FBE4C0E0EBC0E07B057A9879DA1259C7
:0DCC33000015811581120093E4FE7F01229F
:10CC40001200937B057A9879B2125900120093E48E
:10CC5000FEFF2202D0CD904412E004F09044117007
:10CC600003E004F09044101250DD12008AEB90446F
:10CC700010F0A3EAF0A3E9F09044101250DD125036
:10CC800090FF1200A8EF33EF904418F012009F407D
:04CC90000302D01DAE
:10CC9400904418E0B4490302CD205028E0B4450282
:10CCA400805C5012E024BF603814700302CD5B2412
:10CCB400FE603C02CDF9E024B9605214700302CD49
:10CCC4006902CDF9E024B5606214607D24FE70032E
:10CCD40002CD8724FB606324FD700302CD7802CD6E
:01CCE400F956
:10CCE5007404904419F00490441AF002CE0C7410A8
:10CCF500904419F0740490441AF002CE0C7412900A
:10CD05004419F0740490441AF002CE0C7414904443
:10CD150019F0740490441AF002CE0C74169044195C
:10CD2500F0740490441AF002CE0C7418904419F073
:10CD3500740490441AF002CE0C741A904419F074DD
:10CD45000490441AF002CE0CE4904419F074089053
:10CD5500441AF002CE0C7403904419F01490441A4E
:10CD6500F002CE0C7401904419F0740490441AF04A
:10CD750002CE0C7402904419F0740790441AF00224
:09CD8500CE0C904413E4F0A3F07D
:10CD8E00120093904414E075F077A4FB240CF58206
:10CD9E00E43420F5837402C0E0E583C0E0E582C090
:10CDAE00E0EB2400F582E43420F583E0FBE4C0E000
:10CDBE00EBC0E0904413E0C0E0A3E0C0E07B057A56
:10CDCE009879A612590074F92581F581904414E0E2
:10CDDE0004F0B402AB1200937B057A957941125997
:10CDEE0000120093E4FE7F012280131200937B0554
:10CDFE007A9879B2125900120093E4FEFF22904401
:0ACE0E0019E0B40F00400302CF2C1E
:10CE1800120093E490441BF090441AE024FEFBE4D3
:10CE280034FFFAF5F090441BE0FDE4B5F0078BF011
:10CE3800EDB5F001D35055E0FB904419E075F009C9
:10CE4800A4FDE4C0E0EDC0E0904387E075F077A46E
:10CE5800242CF582E43420F583D0E02582F582D0B5
:10CE6800E03583F583EB2582F582E43583F583E0AD
:10CE7800FBE4C0E0EBC0E07B057A9879C612590064
:10CE88001581158190441BE004F0808C90441AE0D1
:10CE9800FBE4C0E0EBC0E0904419E075F009A4FDA4
:10CEA800904387E075F077A4242CF582E43420F5CC
:10CEB80083ED2582F582E43583F583E58224FFFD41
:10CEC800E58334FFFCD0E02DF582D0E03CF583E02B
:10CED800FDE4C0E0EDC0E07B057A9879CC125900FA
:0BCEE80015811581904419E0B4012869
:10CEF300904387E075F077A42401F582E43420F5AC
:10CF030083E0FBE4C0E0EBC0E07B057A9879D112C3
:10CF130059001581158180097B057A967969125923
:09CF230000120093E4FE7F0122DC
:10CF2C00120093904419E0540FFBE4C313CB13CBC2
:10CF3C00EB90441CF0904413E4F0A3F090441AE0FE
:10CF4C0024FEFBE434FFFAF5F0904413E0B5F0084E
:10CF5C008BF0A3E0B5F001D35059904413E0FEA33D
:10CF6C00E0FF90441CE02323FB904387E075F077AF
:10CF7C00A42459F582E43420F583EB2582F582E470
:10CF8C003583F583EF2582F582EE3583F583E0FB5F
:10CF9C00E4C0E0EBC0E07B057A9879C61259001525
:10CFAC00811581904414E004F0904413708EE004D9
:10CFBC00F0808990441AE0FBE4C0E0EBC0E09044C0
:10CFCC001CE02323FD904387E075F077A42459F5EA
:10CFDC0082E43420F583ED2582F582E43583F583F4
:10CFEC00E58224FFFDE58334FFFCD0E02DF582D0F3
:10CFFC00E03CF583E0FDE4C0E0EDC0E07B057A9811
:10D00C0079DA12590015811581120093E4FE7F0123
:01D01C0022F1
:10D01D001200937B057A9879B2125900120093E4AD
:0DD02D00FEFF2202D0CD904413E4F0A3F0EA
:10D03A00120093904414E075F077A4FB24A5F582BE
:10D04A00E43442F5837402C0E0E583C0E0E582C0BF
:10D05A00E0EB2499F582E43442F583E0FBE4C0E096
:10D06A00EBC0E0904413E0C0E0A3E0C0E07B057AA7
:10D07A009879A612590074F92581F581904414E033
:10D08A0004F0B402AB1200937B057A9579411259E8
:10D09A0000120093E4FEFF228029120093904410AC
:10D0AA001250DD125090FD3395E0C0E0EDC0E07BF8
:10D0BA00057A9879E212590015811581120093E4D4
:10D0CA00FEFF22120093904419E0B41000400302BC
:02D0DA00D1E3A0
:10D0DC00E490441BF090441AE024FEFBE434FFFA85
:10D0EC00F5F090441BE0FDE4B5F0078BF0EDB5F0E6
:10D0FC0001D3504DE0FB904419E075F009A4FD906C
:10D10C004387E075F077A424C5F582E43442F583B7
:10D11C00ED2582F582E43583F583EB2582F582E4F7
:10D12C003583F583E0FBE4C0E0EBC0E07B057A9847
:10D13C0079C61259001581158190441BE004F080CA
:10D14C009490441AE0FB904419E075F009A4FDE4B6
:10D15C00C0E0EDC0E0904387E075F077A424C5F5FE
:10D16C0082E43442F583D0E02582F582D0E0358329
:10D17C00F583E58224FFFFE58334FFFEEB2FF58278
:10D18C00E43EF583E0FBE4C0E0EBC0E07B057A987D
:10D19C0079CC12590015811581904419E0B40128FD
:10D1AC00904387E075F077A4249AF582E43442F535
:10D1BC0083E0FBE4C0E0EBC0E07B057A9879D11208
:10D1CC0059001581158180097B057A967969125968
:07D1DC000012009302D2FFD4
:10D1E300904419E0540FFBE4C313CB13CBEB9044EF
:05D1F3001CF030333692
:10D1F80012009390441CE0FBE4C0E0EBC0E09044D4
:10D2080019E0FBE4C0E0EBC0E0904387E0FBE4C03A
:10D21800E0EBC0E07B057A99790112590074FA2590
:10D2280081F581120093E490441BF090441BE0B414
:10D238000201D3505690441BE0FBE4C0E0EBC0E091
:10D2480090441CE02323FD904387E075F077A424E5
:10D25800F2F582E43442F583ED2582F582E43583E4
:10D26800F583D0E02582F582D0E03583F583E0FDB3
:10D27800E4C0E0EDC0E07B057A9879C61259001544
:10D2880081158190441BE004F080A090441CE023A9
:10D2980023FB904387E075F077A424F2F582E43409
:10D2A80042F583EB2582F582E43583F583A3A3A3B6
:10D2B800E0FBE4C0E0EBC0E07B057A9879DA12592C
:0AD2C8000015811581120093802DDE
:10D2D2001200939044101250DD125090FD3395E0ED
:10D2E200ED3395E0C0E0EDC0E07B057A9979281234
:10D2F200590015811581120093E4FEFF2290441318
:10D30200E4F0A304F002E090120093901FFEE49375
:10D31200FE740193FFE4FC7D641254E4ECC0E0ED82
:10D32200C0E0E493FE740193FFE4FC7D641254E4D4
:10D33200EEC0E0EFC0E07B057A997945125900749E
:10D34200FC2581F581120093904413E4F0A304F0CC
:10D3520002E090904412E004F09044117003E00463
:10D36200F09044101250DD12008AEB904410F0A3AA
:10D37200EAF0A3E9F09044101250DD125090FF122F
:10D3820000A8EFFD3395E0FCEF904418F0E024F3A1
:10D39200601224C9605624FE605D24F6700302D434
:04D3A2005802D4B6A3
:10D3A600120093905D52E493FE740193FFE4FC7DBA
:10D3B600641254E4ECC0E0EDC0E0E493FE74019323
:10D3C600FFE4FC7D641254E4EEC0E0EFC0E07B05B0
:10D3D6007A99794512590074FC2581F581120093DA
:10D3E600E4FE7F012202D4C41294C7E4FE7F012228
:10D3F60002D4C4120093904413E4F0A3F0904413B3
:10D40600E0FAA3E02471F582EA3420F583E0FB33E9
:10D4160095E0C0E0EBC0E07B057A9979521259009D
:10D4260015811581904414E004F0B405D09020765F
:10D43600E0FB3395E0C0E0EBC0E07B057A997957D5
:10D4460012590015811581120093E4FE7F01220214
:10D45600D4C4120093904413E4F0A3F0904413E074
:10D46600FAA3E0249CF582EA344CF583E0FB33957D
:10D47600E0C0E0EBC0E07B057A99795212590015BD
:10D48600811581904414E004F0B405D0904CA1E0DD
:10D49600FB3395E0C0E0EBC0E07B057A9979571243
:10D4A600590015811581120093E4FE7F0122800E3A
:10D4B6007F06904418E0FD128FF4E4FEFF229044AC
:10D4C60013E4F0A304F002E090120093904F35E0CD
:10D4D600FBE4C0E0EBC0E07B057A99795D12590068
:10D4E60015811581120093904F36E0FBE4C0E0EB06
:10D4F600C0E07B057A99797212590015811581125F
:10D506000093904F3BE0FBE4C0E0EBC0E07B057A84
:10D51600997987125900158115811200939043BAA3
:10D52600E0FBE4C0E0EBC0E0904F37E0FBE4C0E096
:10D53600EBC0E0E0FBE4C0E0EBC0E07B057A997964
:10D54600A112590074FA2581F5811200939043BC0B
:10D55600E0FBE4C0E0EBC0E0904F38E0FBE4C0E065
:10D56600EBC0E0E0FBE4C0E0EBC0E07B057A997934
:10D57600BD12590074FA2581F5811200939043BBC0
:10D58600E0FBE4C0E0EBC0E0904F39E0FBE4C0E034
:10D59600EBC0E0E0FBE4C0E0EBC0E07B057A997904
:10D5A600DC12590074FA2581F5811200939043B973
:10D5B600E0FBE4C0E0EBC0E0904F3AE0FBE4C0E003
:10D5C600EBC0E0E0FBE4C0E0EBC0E07B057A9979D4
:10D5D600F812590074FA2581F581120093904413CC
:10D5E600E4F0A304F002E0907F497B027A4379EFEE
:10D5F60012F69C5004E4FEFF221200939043EFE0E3
:10D60600FBE4C0E0EBC0E07B057A9A791D12590075
:10D6160015811581120093904413E4F0A304F002DF
:10D62600E090904412E004F09044117003E004F09E
:10D636009044101250DDE004F09044117003E004B1
:10D64600F0125090FF1200A8EF3395E0EF904418C7
:10D65600F0E490441DF0740290443DF0A37444F04D
:10D66600A3741DF0904418E0B44C0302D787501EF3
:10D67600E024BD603D14607324FE700302D72A14B3
:10D68600700302D73C14700302D77502D83DE0241C
:10D69600B0700302D7C024FD700302D7D214700302
:10D6A60002D7E414700302D7F514700302D80602F9
:02D6B600D83D5D
:03D6B800303C24DF
:10D6BB009044B77420FBF07FAE7C447D1D12F85C68
:10D6CB0050217B027A44791D7D057C9A782D125569
:04D6DB00BC02D84C69
:10D6DF007B027A44791D7D057C9A78371255BC02FE
:05D6EF00D84C30372487
:10D6F4009044B77420FBF07FAA7C447D1D12F85C33
:10D7040050217B027A44791D7D057C9A782D12552F
:04D71400BC02D84C2F
:10D718007B027A44791D7D057C9A78371255BC02C4
:10D72800D84C7B027A44791D7D027C4E781A1255BA
:07D73800BC02D84C3038247C
:10D73F009044B77420FBF07FA47C447D1D12F85CED
:10D74F0050217B027A44791D7D057C9A782D1255E4
:04D75F00BC02D84CE4
:10D763007B027A44791D7D057C9A78371255BC0279
:10D77300D84C7B027A44791D7D027C4D78BA1255D0
:07D78300BC02D84C303B242E
:10D78A009044B77420FBF07FA87C447D1D12F85C9E
:10D79A0050217B027A44791D7D057C9A782D125599
:04D7AA00BC02D84C99
:10D7AE007B027A44791D7D057C9A78371255BC022E
:10D7BE00D84C7B027A44791D7D027C4D789A1255A5
:10D7CE00BC02D84C7B027A44791D7D027C4D7819BF
:10D7DE001255BC02D84C7B027A44791D7D027C4ED8
:10D7EE0078BA1255BC80577B027A44791D7D027C33
:0BD7FE004D785A1255BC80463036238F
:10D809009044B77420FBF07FAC7C447D1D12F85C1A
:10D8190050207B027A44791D7D057C9A782D12551A
:10D82900BC80207B027A44791D7D057C9A78371269
:10D8390055BC800F7B027A44791D7D057C9A783826
:10D849001255BC740290443DF0A37444F0A3741DB6
:10D85900F01200937B057A96795612590090443D4F
:10D869001250DD125090640A603790443D1250DD29
:10D87900125090602C90443D1250DDE004F0904429
:10D889003E7003E004F0125090FD3395E0C0E0EDE6
:10D89900C0E07B057A967966125900158115818059
:10D8A900BC7B057A96796912590012009302E090BF
:07D8B900904413E4F0A3F01A
:10D8C000120093904414E075F077A4FB24A5F58230
:10D8D000E43442F5837402C0E0E583C0E0E582C031
:10D8E000E0EB2499F582E43442F583E0FBE4C0E008
:10D8F000EBC0E0904413E0C0E0A3E0C0E07B057A19
:10D900009879A612590074F92581F581904414E0A4
:10D9100004F0B402AB1200937B057A957941125959
:10D9200000120093904413E4F0A304F002E090127C
:10D930000093128292EF600B7B057A9A793C125920
:10D940000080097B057A9A793F12590012009312E0
:10D950008266EF600B7B057A9A7942125900800942
:10D960007B057A9A7946125900120093904F2FE066
:10D97000FBE4C0E0EBC0E0904F2EE0FBE4C0E0EB46
:10D98000C0E0904F27E0FBE4C0E0EBC0E0904F2602
:10D99000E0FBE4C0E0EBC0E0904F25E0FBE4C0E03A
:10D9A000EBC0E0904F24E0FBE4C0E0EBC0E0904F20
:10D9B00023E0FBE4C0E0EBC0E0904F22E0FBE4C0DA
:10D9C000E0EBC0E0904F21E0FBE4C0E0EBC0E09072
:10D9D0004F20E0FBE4C0E0EBC0E07B057A9A794A97
:10D9E00012590074EC2581F58112009330280B7BCD
:10D9F000057A9A797112590080097B057A9A7977AC
:10DA000012590030290B7B057A9A797D12590080D2
:10DA1000097B057A9A7980125900120093303F09E8
:09DA20007F13E4FD128FF480175E
:10DA290030400B7B057A9A798312590080097B056E
:10DA39007A9A7991125900120093904413E4F0A351
:10DA490004F002E090904412E004F0904411700355
:10DA5900E004F09044101250DDE004F0904411709D
:10DA690003E004F0125090FF1200A8EF3395E0EFA5
:10DA7900904418F0E490441DF0740290443DF0A3E2
:10DA89007444F0A3741DF0904418E0B44C0302DB15
:10DA9900AB501EE024BD603814606F24FE70030291
:10DAA900DB4D14700302DB5F14700302DB9902DCA7
:10DAB90051E024B0700302DBE524FD700302DBF7BB
:10DAC90014700302DC0824FE700302DC1902DC5125
:03DAD900303C25B9
:10DADC009044B77420F07FAE7C447D1DE4FB12F8BB
:10DAEC005C50217B027A44791D7D057C9A782D123D
:05DAFC0055BC02DC60D6
:10DB01007B027A44791D7D057C9A78371255BC02D7
:05DB1100DC6030372547
:10DB16009044B77420F07FAA7C447D1DE4FB12F884
:10DB26005C50217B027A44791D7D057C9A782D1202
:05DB360055BC02DC609B
:10DB3B007B027A44791D7D057C9A78371255BC029D
:10DB4B00DC607B027A44791D7D027C4E783A12555B
:07DB5B00BC02DC603038253C
:10DB62009044B77420F07FA47C447D1DE4FB12F83E
:10DB72005C50217B027A44791D7D057C9A782D12B6
:05DB820055BC02DC604F
:10DB87007B027A44791D7D057C9A78371255BC0251
:10DB9700DC607B027A44791D7D027C4D78DA125570
:07DBA700BC02DC60303B25ED
:10DBAE009044B77420F07FA87C447D1DE4FB12F8EE
:10DBBE005C50217B027A44791D7D057C9A782D126A
:05DBCE0055BC02DC6003
:10DBD3007B027A44791D7D057C95781A1255BC0227
:10DBE300DC607B027A44791D7D027C4D787A125584
:10DBF300BC02DC607B027A44791D7D027C4D783A5D
:10DC03001255BC80587B027A44791D7D027C4E7884
:09DC1300DA1255BC8047303624BA
:10DC1C009044B77420F07FAC7C447D1DE4FB12F87B
:10DC2C005C50207B027A44791D7D057C9A782D12FC
:10DC3C0055BC80207B027A44791D7D057C9A78370F
:10DC4C001255BC800F7B027A44791D7D027C4D7885
:10DC5C003A1255BC904413E4F0A3F0740290443D86
:10DC6C00F0A37444F0A3741DF01200937B057A9713
:10DC7C00795712590090443D1250DD125090640AAD
:10DC8C00603790443D1250DD125090602C90443D12
:10DC9C001250DDE004F090443E7003E004F01250AA
:10DCAC0090FD3395E0C0E0EDC0E07B057A96796697
:10DCBC001259001581158180BC7B057A9679691201
:10DCCC00590012009302E090120093904294E0FBF2
:10DCDC00E4C0E0EBC0E0904295E0FBE4C0E0EBC0B8
:10DCEC00E0904296E0FBE4C0E0EBC0E0904297E0AD
:10DCFC00C0E0A3E0C0E07B057A9A799D12590074CC
:10DD0C00F82581F581120093904AFFE075F010A47C
:10DD1C002404F582E4344BF583E0FBE4C0E0EBC073
:10DD2C00E0904AFFE075F010A42403F582E4344B34
:10DD3C00F583E0FBE4C0E0EBC0E0904AFFE075F057
:10DD4C0010A42402F582E4344BF583E0FBE4C0E03C
:10DD5C00EBC0E0904AFFE075F010A42401F582E4DA
:10DD6C00344BF583E0FBE4C0E0EBC0E0904AFFE00D
:10DD7C0075F010A47E002400F582E4344BF583E0AA
:10DD8C00FF7C01E4FD1254A8D0E02FFFD0E03EC090
:10DD9C00E0EFC0E07B057A9A799D12590074F82562
:10DDAC0081F581120093904AFFE075F010A42406CF
:10DDBC00F582E4344BF583E0FBE4C0E0EBC0E07BA0
:10DDCC00057A9A79B2125900158115811200939037
:10DDDC004AFFE0FBE4C0E0EBC0E07B057A9A79B245
:10DDEC0012590015811581120093904AFFE075F0CD
:10DDFC0010A4240AF582E4344BF583E0FBE4C0E084
:10DE0C00EBC0E07B057A9A79B21259001581158125
:10DE1C00120093904AFFE075F010A42408F582E4F8
:10DE2C00344BF583E0FBE4C0E0EBC0E07B057A9A71
:10DE3C0079B2125900158115811200937B057A95E0
:10DE4C007941125900904413E4F0A304F002E090DD
:10DE5C0012009330270B7B057A9A79B61259008001
:10DE6C00097B057A9A79D0125900120093904413C9
:10DE7C00E4F0A304F002E090120093AF4BE4FEFC3C
:10DE8C007D641254A8EEA2E795E0C0E0EEC0E0E499
:10DE9C00C0E0C04A7B057A9A79E912590074FC25D6
:10DEAC0081F581120093AF4EE4FEFC7D641254A800
:10DEBC00EEA2E795E0C0E0EEC0E0E4C0E0C04D7B30
:05DECC00057A9B790AB4
:10DED10012590074FC2581F581120093904413E4DA
:10DEE100F0A304F002E090120093904D39E0FBE4BE
:10DEF100C0E0EBC0E07B057A9B792C1259001581BB
:10DF01001581120093904413E4F0A304F002E09011
:10DF1100120093904276E0FBE4C0E0EBC0E07B05A9
:10DF21007A9B793F12590015811581120093904413
:10DF310013E4F0A304F002E090904412E004F090A6
:10DF410044117003E004F09044101250DDE004F03D
:10DF51009044117003E004F0125090FF1200A8EFFA
:10DF610033EF904418F0E490441DF0740290443D66
:10DF7100F0A37444F0A3741DF0904418E024BA6037
:0EDF81000D24FE601A24F560271460358044DC
:10DF8F007B027A44791D7D027C4E785A1255BC80F3
:10DF9F00427B027A44791D7D027C4D78FA1255BC82
:10DFAF0080317B027A44791D7D027C4D78191255A0
:10DFBF00BC80207B027A44791D7D027C4E78FA1258
:10DFCF0055BC800F7B027A44791D7D057C9A78378A
:10DFDF001255BC904413E4F0A3F0740290443DF04A
:10DFEF00A37444F0A3741DF01200937B057A9B7900
:10DFFF005212590090443D1250DD125090640A6045
:10E00F003790443D1250DD125090602C90443D12D9
:10E01F0050DDE004F090443E7003E004F0125090A5
:10E02F00FD3395E0C0E0EDC0E07B057A967966128E
:10E03F0059001581158180BC7B057A967969125933
:10E04F0000120093803B1200939044101250DD1287
:10E05F005090FD3395E0C0E0EDC0E0125090FB33DF
:10E06F0095E0EB3395E0C0E0EBC0E07B057A9B7960
:10E07F006112590074FC2581F581120093E4FEFFB3
:0AE08F0022904413E0FEA3E0FF22FC
:10E09900904465EBF0A3EAF0A3E9F09044651250CF
:10E0A900DDE004F09044667003E004F0125090FF44
:10E0B9001200A8EF9043F4F0645B6022E06480B43E
:10E0C900C100400C9043F4E06480B4C401D3400E15
:10E0D9007F239043F4E0FD128FF4E4FEFF22904386
:10E0E900F4E0B45B129044651250DD125090FF12B7
:10E0F90000A8EF9043F4F0E49043F5F09043F4E086
:0FE1090024BF600B14601814600D14601A80207E
:10E1180074019043F5F0802674059043F5F0801E55
:10E1280074FF9043F5F0801674FB9043F5F0800E71
:10E138007F239043F4E0FD128FF4E4FEFF22904227
:10E1480077E014601214607514700302E22A1470E8
:07E158000302E28C02E2E287
:10E15F009042CEE09043F3F0B4FF0B9043F5E064B0
:10E16F0001700302E2E29043F3E0B4FB00400B9036
:10E17F0043F5E06405700302E2E29043F3E0700AB6
:10E18F009043F5E0F4700302E2E29043F3E0B4044D
:0FE19F0001D3500B9043F5E064FB700302E2E202
:10E1AE009043F5E0FA9043F3E02AF07F01E4FDE0BE
:10E1BE00FB1286E602E2E29042CFE09043F3F0B427
:10E1CE00FF0B9043F5E06401700302E2E29043F32B
:10E1DE00E0B4FB00400B9043F5E06405700302E2EF
:10E1EE00E29043F3E0700A9043F5E0F4700302E22C
:10E1FE00E29043F3E0B40401D3500B9043F5E06496
:06E20E00FB700302E2E2D6
:10E214009043F5E0FA9043F3E02AFBF07F017D019F
:10E224001286E602E2E29042D7E09043F3F0B4FFB4
:10E234000B9043F5E06401700302E2E29043F3E0E3
:10E24400B4FB00400B9043F5E06405700302E2E286
:10E254009043F3E0700A9043F5E0F4700302E2E2C5
:10E264009043F3E0B40401D350089043F5E064FB19
:02E27400606CDC
:10E276009043F5E0FA9043F3E02AF07F02E4FDE0F4
:10E28600FB1286E680569042D8E09043F3F0B4FF46
:10E29600089043F5E0640160439043F3E0B4FB006B
:10E2A60040089043F5E0640560329043F3E0700760
:10E2B6009043F5E0F460259043F3E0B40401D350B5
:09E2C600089043F5E064FB6013CD
:10E2CF009043F5E0FA9043F3E02AFBF07F027D01E3
:10E2DF001286E61200939043F3E0FBE4C0E0EBC03C
:10E2EF00E07B057A9B798E125900158115811200FA
:06E2FF0093E4FE7F012202
:10E30500904465EBF0A3EAF0A3E9F0125090FF12F8
:0DE3150000A8EF24BD603B24F06002806A88
:10E32200D2427401904277F07B057A9879A412590F
:10E33200001200939042CEE0FB9043F6F0E4C0E07E
:10E34200EBC0E07B057A9B79951259001581158106
:10E352001200938048D2427402904277F07B057A91
:10E362009879A41259001200939042CFE0FB904397
:10E37200F6F0E4C0E0EBC0E07B057A9B79AB125982
:10E3820000158115811200938013C242E4904277F6
:10E39200F07B057A95799E125900120093E4FE7F74
:02E3A200012256
:10E3A400EBFDEAFCE9F8125090B420001282BAEFB7
:02E3B400600007
:10E3B6001200937B057A957941125900120093E475
:04E3C600FE7F0122B3
:10E3CA00904465EBF0A3EAF0A3E9F0125090FF1233
:04E3DA00009C503320
:10E3DE009044651250DD125090540F904275F0C467
:10E3EE0054F0FAE04AFDF07F4812F17A400302E45D
:01E3FE009D81
:10E3FF001200937B057A9B79C31259001200930286
:02E40F00E49D8A
:10E411009044651250DD125090FF1200A8EF24AC19
:08E42100600B24FC6002804F37
:0CE4290012F09C806F904275E0B455200A
:09E435007F48E0FD12F17A500F5E
:10E43E001200937B057A9B79C312590012009374D4
:07E44E00AA904275F080481E
:0CE455007F48904275E0FD12F17A500FF4
:10E461001200937B057A9B79C312590012009374B1
:10E4710055904275F080251200939044651250DD4D
:10E48100125090FD3395E0C0E0EDC0E07B057A9B32
:10E4910079D4125900158115811200931200937BD2
:10E4A100057A957941125900120093E4FE7F012209
:10E4B100904465EBF0A3EAF0A3E9F0125090FF124B
:10E4C10000A89044651250DDEF1250499044651246
:10E4D10050DDE004F09044667003E004F0125090C7
:0BE4E10024BC600724FC604F02E581B2
:10E4EC009044651250DD125090FF1200A8904465C4
:10E4FC001250E6EF12502D12506524D060051460B6
:03E50C0010801567
:10E50F00C219128BBFC231C218128B728078D21807
:10E51F00128B7280717F069044651250DD125090FD
:10E52F00FD33128FF4E4FEFF229044651250DD128A
:10E53F005090FF1200A89044651250E6EF12502D34
:0CE54F0012506524D0600514600B80128F
:10E55B00C219128BBFC2318031D219128BBFD2318B
:10E56B0080287F069044651250DD125090FD3312C7
:10E57B008FF4E4FEFF227F069044651250DD1250AB
:10E58B0090FD33128FF4E4FEFF221200939044654A
:10E59B001250DD125090FD3395E0C0E0EDC0E07BF2
:10E5AB00057A95794112590015811581120093E472
:04E5BB00FE7F0122BC
:10E5BF00904465EBF0A3EAF0A3E9F01200939044C6
:10E5CF00651250DDE004F09044667003E004F01231
:10E5DF005090FF1200A8EF9043F7F0640A6004E038
:03E5EF00B40D0A5E
:10E5F2007F011293FDE4FE7F01229043F7E024B7EE
:05E60200600302E68D3B
:10E607009044651250DD120087EF9043F8F012F145
:0BE617000FE433FE904468F0B40120D3
:10E622009043F8E0FBE4C0E0EBC0E07B057A9B7925
:10E63200EE12590015811581120093E4FE7F01222A
:07E64200904468E0B4021FE0
:10E649009043F8E0FBE4C0E0EBC0E07B057A9C79FD
:10E659000212590015811581120093E4FEFF2290E0
:05E669004468E0701E92
:10E66E009043F8E0FBE4C0E0EBC0E07B057A9C79D8
:10E67E001612590015811581120093E4FEFF221225
:10E68E0000937B057A9C792A125900120093E4FEBE
:02E69E00FF2259
:10E6A000904465EBF0A3EAF0A3E9F0125090331226
:10E6B00000939042CEE0FBE4904468F0A3EBF0902E
:10E6C00042CFE0FBE490446AF0A3EBF090446AE0B0
:10E6D000C0E0A3E0C0E0904468E0C0E0A3E0C0E098
:10E6E0007B057A9C794112590074FC2581F5819053
:10E6F00042D7E0FBE4904468F0A3EBF09042D8E00E
:10E70000FBE490446AF0A3EBF012009390446AE0BB
:10E71000C0E0A3E0C0E0904468E0C0E0A3E0C0E057
:10E720007B057A9C795512590074FC2581F5817F0F
:09E73000011293FDE4FE7F0122B9
:0EE73900125090B42000C22312799E30231398
:10E747001200937B057A95799E125900120093E483
:03E75700FEFF22A0
:0AE75A007F011293FDE4FE7F01220F
:10E76400904465EBF0A3EAF0A3E9F0125090FF1295
:0DE7740000A8EF24BD603B24F06002806A25
:10E78100D2427403904277F07B057A9879A41259AA
:10E79100001200939042D7E0FB9043F9F0E4C0E00F
:10E7A100EBC0E07B057A9C796912590015811581CE
:10E7B1001200938048D2427404904277F07B057A2C
:10E7C1009879A41259001200939042D8E0FB90432B
:10E7D100F9F0E4C0E0EBC0E07B057A9C797D125949
:10E7E10000158115811200938013C242E490427793
:10E7F100F07B057A95799E125900120093E4FE7F11
:02E801000122F2
:10E80300904465EBF0A3EAF0A3E9F090422FE0FA1D
:10E81300A3E0FB904231EAF0A3EBF090422FE0FA41
:10E82300A3E0FB904233EAF0A3EBF090446512506F
:10E83300DD125090FF1200A8EF9043FAF090446766
:10E84300E004F09044667003E004F09044651250D5
:10E85300DD12008AEB904465F0A3EAF0A3E9F0909F
:10E8630043FAE024BE601514605124FE606024F274
:0CE87300700302E91124FC607F02E957E9
:10E87F009044651250DD120087EE9043FBF0A3EF3A
:0CE88F00F09043FBE0B40102A3E0501045
:10E89B009043FCE0FA904231125499EAF002E96A93
:10E8AB001200937B057A95799E125900120093E41E
:10E8BB00FEFF229044651250DD90423112549912A2
:10E8CB005090F002E96A9044651250DD120087EE19
:10E8DB009043FBF0A3EFF090422FE0FCA3E0FD127E
:05E8EB00945FEF607A6C
:10E8F0007F08E4FD128FF4E4FEFF2290446512507D
:10E90000DD120087904233125499EEF0A3EFF080AD
:10E91000599044651250DD125090640A604C904446
:10E92000651250DD12509060419044651250DDE058
:10E9300004F09044667003E004F0904231E0FCA3E0
:10E94000E0FDE004F09042317003E004F08C838D30
:10E9500082125090F080BA1200937B057A95799ECE
:10E96000125900120093E4FEFF221200937B057AF5
:0EE970009C7993125900120093E4FE7F01225D
:10E97E00904465EBF0A3EAF0A3E9F0904D39E03056
:02E98E00E42C77
:10E990001200937B057A9C79961259001200937BA2
:10E9A000057A9C79C81259001200937B057A9C79EC
:10E9B000F8125900120093E4FE7F0122C224C2081B
:10E9C0009044651250DD125090FF1200A24004E402
:10E9D000FFFE229044651250DD125090FF1200A8F5
:10E9E0009044651250E6EF12502DC22BC22C1250EB
:10E9F0006524BD600E24FD602C24F6602C24F86094
:03EA000051802A18
:10EA03001200937B057A9D791E125900120093C25E
:10EA1300AF75A80075A70075A5E175A51E758702DA
:10EA2300802DD22B8029D22C80251200939044650F
:10EA33001250DD125090FD3395E0C0E0EDC0E07B55
:10EA4300057A9D792C1259001581158112009320A6
:0DEA53002B06202C0302EB24E4904468F015
:05EA6000E4904469F0A0
:10EA6500302B55904468E0C0E0904469E0FDE0FB40
:10EA7500E4C0E0EBC0E0904468E075F009A4FFE471
:10EA8500C0E0EFC0E0904387E075F077A4242CF553
:10EA950082E43420F583D0E02582F582D0E0358309
:10EAA500F583D0E02582F582D0E03583F583E0FB60
:10EAB500D0E0FF1286E6804B904468E0C0E09044C9
:10EAC50069E0FDE0FB904468E075F009A4FFE4C04F
:10EAD500E0EFC0E0904387E075F077A42457F58216
:10EAE500E4344CF583D0E02582F582D0E03583F51A
:10EAF50083EB2582F582E43583F583E0FBD0E0FFE7
:10EB05001286E6904469E004F0B40802800302EA44
:10EB150065904468E004F0B40502800302EA607F72
:08EB2500011293FDE4FEFF2242
:10EB2D0041444452203078253034582C20444154EF
:10EB3D00412030782530325820230A005361766504
:0FEB4D006420256420230A0009256420210A0082
:10EB5C00740290445FF0A37441F0A3747EF090446F
:10EB6C005F1250DD12008AEB90445FF0A3EAF0A331
:10EB7C00E9F090445F1250DD125090FF1200A8EFA4
:0AEB8C009043FDF020420302ED2B40
:09EB9600E0B40D02800302EC64FE
:10EB9F00C242904277E014600B14601C14602D1475
:04EBAF00603E804EF6
:10EBB3009043FF744CF0A37460F09042CEE0904316
:10EBC300FEF0803A9043FF744CF0A37461F09042DE
:10EBD300CFE09043FEF080269043FF744CF0A37483
:10EBE30069F09042D7E09043FEF080129043FF74A7
:10EBF3004CF0A3746AF09042D8E09043FEF0904347
:10EC0300FEE0FF9043FFE0FCA3E0FD12945FEF60A2
:01EC13002AD6
:10EC14009043FEE0FBE4C0E0EBC0E09043FFE0C0C3
:10EC2400E0A3E0C0E07B057AEB792D12590074FC77
:10EC34002581F5811200937F0122E4904277F0123E
:10EC440000939043FEE0FBE4C0E0EBC0E07B057A78
:10EC5400EB794912590015811581120093E4FF22C2
:0DEC64009043FDE0FF120099400302ED0512
:10EC710090445F1250DD120087EE9043FFF0A3EF46
:10EC8100F09043FFE0B40006A3E0B4FF01D350715C
:10EC9100904400E09043FEF0904277E014600B1442
:0AECA100601614602114602C803608
:10ECAB007F01E4FD9043FEE0FB1286E680287F01A6
:10ECBB007D019043FEE0FB1286E6801A7F02E4FDA5
:10ECCB009043FEE0FB1286E6800C7F027D019043B1
:10ECDB00FEE0FB1286E61200939043FEE0FBE4C0DD
:10ECEB00E0EBC0E07B057AEB7955125900158115E5
:10ECFB0081120093E4FF22E4FF229043FDE0B41B5A
:01ED0B0018EF
:10ED0C00904461E004F09044607003E004F090449F
:10ED1C005F1250DD12E09922C242E4904277F090EB
:10ED2C0043FDE0B4470302EF005052E0B43F03024E
:10ED3C00EE925025E0700302EDF124F6700302ED23
:10ED4C00E424FD700302EDDC24F2700302EDFE24DA
:10ED5C00E1700302EE5F02F044E024BF700302EEA8
:10ED6C002914700302EE4414700302EEAD14700308
:10ED7C0002EEC824FE700302EEE302F044E0B4524B
:10ED8C000302EFA25025E024B8700302EF1B1470AD
:10ED9C000302EF3624FD700302EF5114700302EFEF
:10EDAC006C24FD700302EF8702F044E024AC700386
:10EDBC0002EFBD24FE700302EFD814700302EFF3D0
:10EDCC0014700302F00E24FE700302F02902F044CA
:10EDDC007F011293FD7F01227F229043FDE0FD1203
:10EDEC008FF47F01227F229043FDE0FD128FF47F90
:05EDFC00012220420D80
:10EE01007F229043FDE0FD128FF47F012290446147
:10EE1100E004F09044607003E004F090445F12500D
:10EE2100DD12008A12E09922904461E004F09044DE
:10EE3100607003E004F090445F1250DD12008A120A
:10EE41009D5D22904461E004F09044607003E00411
:10EE5100F090445F1250DD12008A129E11229044FC
:10EE610061E004F09044607003E004F090445F12AC
:0CEE710050DD12008A12006FEE4F700A94
:0DEE7D007F15E4FD128FF4E4FF222005074D
:10EE8A007F041293FD7F0122904461E004F09044D4
:10EE9A00607003E004F090445F1250DD12008A12A1
:10EEAA00E6A022904461E004F09044607003E0041C
:10EEBA00F090445F1250DD12008A129F042290449F
:10EECA0061E004F09044607003E004F090445F1243
:10EEDA0050DD12008A12C35222904461E004F0907D
:10EEEA0044607003E004F090445F1250DD12008A1F
:10EEFA001250277F0122904461E004F09044607030
:10EF0A0003E004F090445F1250DD12008A12007B85
:10EF1A0022904461E004F09044607003E004F090B1
:10EF2A00445F1250DD12008A12E30522904461E028
:10EF3A0004F09044607003E004F090445F1250DDE6
:10EF4A0012008A12E3A422904461E004F090446023
:10EF5A007003E004F090445F1250DD12008A12E35D
:10EF6A00CA22904461E004F09044607003E004F027
:10EF7A0090445F1250DD12008A12E4B1229044617B
:10EF8A00E004F09044607003E004F090445F125093
:10EF9A00DD12008A12E5BF22904461E004F0904439
:10EFAA00607003E004F090445F1250DD12008A1290
:10EFBA00008122904461E004F09044607003E00410
:10EFCA00F090445F1250DD12008A12E73922904411
:10EFDA0061E004F09044607003E004F090445F1232
:10EFEA0050DD12008A12E76422904461E004F09036
:10EFFA0044607003E004F090445F1250DD12008A0E
:10F00A0012E80322904461E004F09044607003E047
:10F01A0004F090445F1250DD12008A12502A2290A6
:10F02A004461E004F09044607003E004F090445FAF
:10F03A001250DD12008A12E97E227F069043FDE01B
:07F04A00FD128FF47F01228B
:10F051009044CCEFF09044CDEDF0E49044CEF090AC
:10F0610044CCE0F5F09044CEE0B5F000502CE490B3
:10F0710044CFF09044CFE0FAE004F0EA60141200CB
:10F08100969044CDE0F5F09044CFE0B5F00050E328
:0BF0910080E19044CEE004F080C52236
:10F09C007480903F01F07453903F00F074A0903F47
:0FF0AC0001F0741C903F00F074C1903F01F022FE
:06F0BB00EF903F01F0227E
:06F0C100EF903F00F02279
:06F0C700903F00E0FF2273
:06F0CD00903F01E0FF226C
:10F0D300903F01E0904401F0E4904402F090440139
:04F0E300E020E02722
:10F0E700120096903F01E0904401F0904402E0B492
:04F0F7000A00400BC0
:10F0FB0074C3903F01F0E4904402F0904402E004AA
:04F10B00F080D2229C
:10F10F009044CCEFF012F0D39044CCE0FF12F0C15A
:10F11F007FC512F0BBE4904404F012F0CDEF9044A1
:10F12F0003F0EF54806016904404E0B40300500DD8
:03F13F00302DE789
:10F14200904404E004F0C22D80DD904404E0B40356
:03F1520000400A70
:10F155007FC312F0BB12F0D3D322904403E030E317
:01F165000A9F
:10F166007FC312F0BB12F0D3C3227FC312F0BB12CF
:04F17600F0D3D322DD
:10F17A009044ECEFF09044EDEDF012F0D39044ECB3
:10F18A00E0903F00F012009674C5903F01F0E490C1
:10F19A004405F0903F01E09044EEF05480601690F0
:08F1AA004405E0B40300500D20
:03F1B200302DE815
:10F1B500904405E004F0C22D80DE9044EEE0540852
:0BF1C5007009904405E0B40300400B0B
:10F1D00074C3903F01F012F0D3D3229044EDE0903D
:10F1E0003F00F0E4904405F0903F01E09044EEF0E1
:0DF1F00054806016904405E0B40300500DFB
:03F1FD00302DE8CA
:10F20000904405E004F0C22D80DE9044EEE0540806
:0BF210007009904405E0B40300400BBF
:10F21B0074C3903F01F012F0D3D32274C3903F011B
:06F22B00F012F0D3C32233
:10F231009044ECEFF09044EDEDF09044EEEBF012E1
:10F24100F0D39044ECE0903F00F074C5903F01F0A2
:10F25100E4904406F0903F01E09044EFF054806068
:0AF2610016904406E0B40300500DBF
:03F26B00302DE85B
:10F26E00904406E004F0C22D80DE9044EFE0540896
:0BF27E007009904406E0B40300400B50
:10F2890074C3903F01F012F0D3D3229044EDE09083
:10F299003F00F0E4904406F0903F01E09044EFF025
:0DF2A90054806016904406E0B40300500D40
:03F2B600302DE810
:10F2B900904406E004F0C22D80DE9044EFE054084B
:0BF2C9007009904406E0B40300400B05
:10F2D40074C3903F01F012F0D3D3229044EEE09037
:10F2E4003F00F0E4904406F0903F01E09044EFF0DA
:0DF2F40054806016904406E0B40300500DF5
:03F30100302DE8C4
:10F30400904406E004F0C22D80DE9044EFE05408FF
:0BF314007009904406E0B40300400BB9
:10F31F0074C3903F01F012F0D3D32274C3903F0116
:06F32F00F012F0D3C3222E
:10F335009044DAEFF09044DBEBF0A3EAF0A3E9F0B8
:10F34500E4904407F012F0D39044DAE0903F00F0E7
:10F3550074C5903F01F09044D9E0F5F0904407E082
:05F36500B5F000503678
:08F36A00903F01E0FF30E702D3
:06F3720080F6EF30E30815
:10F3780074C3903F01F0D322904407E004F0904416
:10F38800DB1250DDE004F09044DC7003E004F0127E
:10F398005090903F00F080BB903F01E0FF30E702C3
:0AF3A80080F674C3903F01F0C32209
:10F3B2009044DFEFF09044E0EBF0A3EAF0A3E9F031
:10F3C200E4904408F012F0D39044DFE0903F00F064
:10F3D20074C5903F01F09044DEE024FFFBE434FF6B
:10F3E200F5F0904408E0FDE4B5F0068BF0EDB5F0E1
:03F3F20000505870
:08F3F500903F01E0FE30E70249
:06F3FD0080F6EE30E3286B
:10F4030074C3903F01F0903F00E0FC9044E0125041
:10F41300DDE004F09044E17003E004F0EC125049A5
:10F42300904408E004FFF022904408E004F0903F89
:10F4330000E0FC9044E01250DDE004F09044E17001
:10F4430003E004F0EC125049808B7440903F01F0CC
:10F45300904408E004F0903F00E0FC9044E0125038
:10F46300DDE004F09044E17003E004F0EC12504955
:08F47300903F01E0FE30E702CA
:10F47B0080F674C3903F01F0904408E004F0903F95
:10F48B0000E0FC9044E01250DDE004F09044E170A9
:0BF49B0003E004F0EC125049E4FF22F3
:10F4A6009044E3EFF09044E4ECF0A3EDF012F0D3D7
:10F4B6009044E3E0903F00F074C5903F01F012F0F5
:07F4C600CDEFFEEF30E7027D
:06F4CD0080F5EE30E315AE
:10F4D300903F00E0FA9044E4125499EAF07FC3129B
:05F4E300F0BB7F0122D7
:10F4E800903F00E0FA9044E4125499EAF074C39013
:10F4F8003F01F0903F00E0FA9044E4125499EAF09A
:09F5080074C3903F01F0E4FF22FE
:10F511009044C5EFF09044C6EBF0A3EAF0A3E9F004
:10F5210012F0D39044C5E0903F00F07F017D1412AA
:10F53100F05174C5903F01F07F017D1412F051909C
:0AF541003F01E09044C9F030E702FA
:09F54B0080F39044C9E030E308AC
:10F5540074C3903F01F0D3227444903F00F0903F75
:09F5640001E09044C9F030E70217
:09F56D0080F39044C9E030E3088A
:10F5760074C3903F01F0D3227F017DFF12F05174D6
:10F58600C3903F01F07F0A7DFF12F05112F0D39035
:10F5960044C5E04401903F00F07F017D1412F05114
:10F5A60074C5903F01F07F017D1412F051903F0128
:08F5B600E09044C9F030E702C7
:09F5BE0080F39044C9E030E30839
:10F5C70074C3903F01F0D3227F047DFF12F05112E4
:0CF5D700F0C7EFFE903F01E0FE30E702BD
:06F5E30080F6EE30E308A3
:10F5E90074C3903F01F0D3227F017DFF12F05112C5
:0CF5F900F0C7EF9044C9F0E49044CAF061
:0BF60500903F01E09044C9F030E702A4
:09F6100080F39044C9E030E308E6
:10F6190074C3903F01F0D3229044CAE0B402067447
:10F6290040903F01F0903F00E0FF9044C61250E641
:10F639009044CAE0FBE82BFEE43CFCEEF8EF1250E4
:10F649002D7F047DFF12F0519044CAE004F0B40309
:08F65900AB903F01E030E70235
:10F6610080F774C3903F01F0903F00E0FC9044C6E6
:10F671001250DDECC0E074031250C5D0E0125049C5
:05F6810012F0D3C322CA
:10F686009044C5EFF09044C6EDFBF07D4012F23198
:06F696005002D322C32242
:10F69C009044B7EFF09044B8EBF0A3EAF0A3E9F094
:10F6AC0012F0D39044B7E0903F00F074C5903F0146
:09F6BC00F0903F01E0FE30E7028E
:06F6C50080F6EE30E30BBD
:10F6CB0074C3903F01F012F0C7D32212F0C7EFFEC4
:08F6DB00903F01E0FE30E70260
:06F6E30080F6EE30E30B9F
:10F6E90012F0C774C3903F01F0D3227F4012F0BBE0
:10F6F90012F0C79044B81250DDEF12504974C3900C
:08F709003F01F012F0C7C3221A
:10F711009044E6EFF09044E7EDF012F17A5002D315
:03F7210022C322DE
:10F72400696E2077726974655F383538315F627944
:10F7340074652C2074696D6564206F757420617420
:10F744002025642077616974696E6720666F722072
:10F75400646576696365202530325820746F2062B1
:10F7640065636F6D6520617661696C61626C6521AA
:02F774000A0089
:10F776009044C5EFF09044C6EDF09044C7EBF0908E
:10F786004409E4F0A3F0904409E0B42705A3E0B4EB
:10F796001000501A9044C5E0FF12F10F401090443B
:10F7A6000AE004F090440970DDE004F080D890444B
:0CF7B60009E0B42705A3E0B41000402FC8
:10F7C2001200933033249044C5E0FBE4C0E0EBC068
:10F7D200E0904409E0C0E0A3E0C0E07B057AF7795D
:10F7E2002412590074FC2581F581120093D3221250
:10F7F200F0D39044C5E0903F00F074C5903F01F013
:08F80200903F01E0FB30E7023A
:06F80A0080F6EB30E3087C
:10F8100074C3903F01F0D3229044C6E0903F00F0C3
:08F82000903F01E0FB30E7021C
:06F8280080F6EB30E3085E
:10F82E0074C3903F01F0D3229044C7E0903F00F0A4
:08F83E00903F01E0FB30E702FE
:06F8460080F6EB30E30840
:10F84C0074C3903F01F0D32274C3903F01F0C322E4
:10F85C009044B8EFF09044B9ECF0A3EDF0EF54FE07
:10F86C009044BBF0EB547FFDE490440BF0A3EDF01F
:0FF87C009044BBE0FF90440CE0FD12F17A500283
:10F88B00D3229044B8E04401903F00F074C5903F00
:0DF89B0001F0903F01E09044BBF030E70227
:09F8A80080F39044BBE030E3085A
:10F8B10074C3903F01F0D32212F0C7EF9044BBF024
:0BF8C100903F01E09044BBF030E702F4
:09F8CC0080F39044BBE030E30836
:10F8D50074C3903F01F0D3227F017DFF12F0519058
:10F8E500440BE4F0A3F090440BE0FCA3E0FD90444E
:10F8F500B7E0FB75F000ECBC00068BF0EDB5F00051
:02F9050050723E
:0BF90700903F01E09044BBF030E702AD
:09F9120080F39044BBE030E308EF
:10F91B0074C3903F01F0D32290440BE0FCA3E0FDB5
:10F92B009044B7E024FFFBE434FFF5F0ECB5F00CAA
:10F93B008BF0EDB5F0067440903F01F0903F00E086
:10F94B00FC9044B9E0FAA3E0FBE004F09044B970FA
:10F95B0003E004F08A838B82ECF090440CE004F01B
:10F96B0090440B600302F8EBE004F002F8EB903FDD
:05F97B0001E030E7028D
:10F9800080F774C3903F01F0903F00E0FA9044B9D3
:0AF99000125499EAF012F0D3C322DA
:09F99A007766210A0050460A00BC
:10F9A30075A70075A880D2ACE490444DF0303612B0
:10F9B300E4FF7D01E4FB1286E6E4FFE4FDE4FB12D1
:10F9C30086E63037077F4C7DFE12F711E4F533E40A
:10F9D300F534E534FB7A00EB2480F582EA3440F514
:10F9E30083E4F0740190444DF0904AFFE0FAEA900A
:10F9F300444EF0904B0090444EE075F010A4FB7A17
:10FA03000074052BF8744B3AF5838882E0FAEA9088
:10FA13004444F0904B0090444EE075F010A4FB7A00
:10FA23000074062BF8744B3AF5838882E0FAEA9067
:10FA33004445F090444EE075F010A4FB7A00904BDF
:10FA430000EB2400F8EA344BF5838882E0FAEA906D
:10FA53004449F0904B0090444EE075F010A4FB7ABB
:10FA63000074012BF8744B3AF5838882E0FAEA902C
:10FA7300444AF0904B0090444EE075F010A4FB7A9A
:10FA83000074022BF8744B3AF5838882E0FAEA900B
:10FA93004446F0904B0090444EE075F010A4FB7A7E
:10FAA3000074032BF8744B3AF5838882E0FAEA90EA
:10FAB3004447F0904B0090444EE075F010A4FB7A5D
:10FAC3000074042BF8744B3AF5838882E0FAEA90C9
:10FAD3004448F0904B0090444EE075F010A4FB7A3C
:10FAE3000074072BF8744B3AF5838882E0FAEA90A6
:10FAF300444BF0904B0090444EE075F010A4FB7A19
:10FB03000074082BF8744B3AF5838882E0FAEA9084
:0AFB1300444CF0904445E0B4FF0DAF
:10FB1D009044441250D4E4904445F08006904445FE
:10FB2D001250D4E4FA90444AE02A904298FAE02A1E
:10FB3D00904443F0904294E0FA904448E02A904477
:10FB4D0048F0904295E0FA904447E02A904447F0FF
:10FB5D00904296E0FA904446E02A904446F0904454
:07FB6D0048E0B43C00401029
:10FB7400904448E024C4904448F09044471250D440
:09FB8400904447E0B43C0040103D
:10FB8D00904447E024C4904447F09044461250D42A
:09FB9D00904446E0B41800401049
:10FBA600904446E024E8904446F09044431250D4F2
:07FBB60090444CE0B4FF0D88
:10FBBD00E490444CF090444B1250D4800690444C49
:10FBCD001250D4904443E0FB7A00EB5400FBEA540E
:10FBDD00FFFAEAFBE4FAEB904449F0904443E0FB72
:10FBED007A00EB54FFFBEA5400FAEB90444AF09094
:10FBFD00444EE075F010A4FB7A00904B00EB24000E
:10FC0D00FBEA344BFA90444FEAF0A3EBF0904449F1
:10FC1D00E0FF90444FE0FCA3E0FD120066EE4F6064
:10FC2D0005E490444DF0904B0090444EE075F0107B
:10FC3D00A4FB7A0074012BFB744B3AFA90444FEA03
:10FC4D00F0A3EBF090444AE0FF90444FE0FCA3E0BA
:10FC5D00FD120066EE4F6005E490444DF0904B00B0
:10FC6D0090444EE075F010A4FB7A0074022BFB74E7
:10FC7D004B3AFA90444FEAF0A3EBF0904446E0FF84
:10FC8D0090444FE0FCA3E0FD120066EE4F6005E4EA
:10FC9D0090444DF0904B0090444EE075F010A4FB55
:10FCAD007A0074032BFB744B3AFA90444FEAF0A39D
:10FCBD00EBF0904447E0FF90444FE0FCA3E0FD12D1
:10FCCD000066EE4F6005E490444DF0904B0090447B
:10FCDD004EE075F010A4FB7A0074042BFB744B3AC4
:10FCED00FA90444FEAF0A3EBF0904448E0FF9044C3
:10FCFD004FE0FCA3E0FD120066EE4F6005E490447A
:10FD0D004DF0904B0090444EE075F010A4FB7A003E
:10FD1D0074052BFB744B3AFA90444FEAF0A3EBF0C9
:10FD2D00904444E0FF90444FE0FCA3E0FD120066D8
:10FD3D00EE4F6005E490444DF0904B0090444EE042
:10FD4D0075F010A4FB7A0074062BFB744B3AFA90F5
:10FD5D00444FEAF0A3EBF0904445E0FF90444FE0B0
:10FD6D00FCA3E0FD120066EE4F6005E490444DF0FB
:10FD7D00904B0090444EE075F010A4FB7A00740790
:10FD8D002BFB744B3AFA90444FEAF0A3EBF09044FE
:10FD9D004BE0FF90444FE0FCA3E0FD120066EE4FF8
:10FDAD006005E490444DF0904B0090444EE075F0AA
:10FDBD0010A4FB7A0074082BFB744B3AFA90444F55
:10FDCD00EAF0A3EBF090444CE0FF90444FE0FCA32D
:10FDDD00E0FD120066EE4F6005E490444DF0904456
:04FDED004DE0700E67
:0EFDF1001200937B057AF9799A125900800C62
:10FDFF001200937B057AF9799F125900120093C272
:10FE0F00AF75A80075A70075A5E175A51E758702CA
:01FE1F0022C0
:03FE20000549226F
:03FE2300054C2269
:0EFE2600C2CF75A61E75A6E11551E5517005F7
:09FE3400755164D200759710228B
:10FE3D00759700858452E55390427EF0859453E585
:10FE4D0054904281F085A45485B45585C45785D40A
:07FE5D005885E459D22D2263
:04FE640012009622D0
:04FE680012009622CC
:04FE6C0012009622C8
:04FE700012009622C4
:04FE740012009622C0
:04FE780012009622BC
:04FE7C0012009622B8
:10FE800090440DEBF0A3EAF0A3E9F0EDFB7A00EB70
:10FE9000FAE4FB904451EAF0A3EBF0904451E0FC0B
:10FEA000A3E0FD90440D1250CB09B900010A125095
:10FEB00090FEEDC39EFD19C0D0B9FF011AD0D0123B
:10FEC0005090F8EC98FC904451ECF0A3EDF0904485
:10FED00052E0FB904451E0FA75F005EAA2E713CB3B
:10FEE00013CBD5F0F7FA904451EAF0A3EBF090442D
:10FEF00051E0FCA3E0FD90440D1250CB09B9000184
:10FF00000A1250902DFD19C0D0B9FF011AD0D0129D
:10FF100050903CFC90440D1250CBEC1250BBED12B3
:03FF200050492223
:01FFF000AA66
:01FFF10055BA
:01FFF200FF0F
:02FFF3005000BC
:02FFF500EFF922
:01FFF7007E8B
:00000001FF
